S31508001800B00A0020D9180008E7180008E9180008E7
S3150800181000000000000000000000000000000000BA
S315080018200000000000000000000000000119000888
S31508001830000000000000000003190008013C000831
S31508001840994C000807190008071900080719000825
S3150800185007190008071900080719000807190008DA
S31508001860071900089D290008071900080719000824
S3150800187007190008071900080719000807190008BA
S3150800188007190008000000000000000007190008FA
S3150800189000000000071900080719000807190008C2
S315080018A00000000007190008071900088D45000800
S315080018B007190008071900080719000800000000A2
S315080018C0EE11AA550348854600F006FD0048004774
S315080018D0B17A0008B00A00200B4880F308880B4844
S315080018E080470B480047FEE704207146084202D0AD
S315080018F0EFF3098001E0EFF30880714605F024FF55
S31508001900FEE7FEE7FEE7FEE7B00A0020B93E00085C
S31508001910C518000830B50B460146002020220124D0
S3150800192009E00D46D5409D4205D31D469540491B05
S315080019302546954040191546521E002DF1DC30BD4E
S3150800194070B500242546002801DA01244042002902
S3150800195001DA01254942FFF7DDFFAC4200D04042DB
S31508001960002C00D0494270BD03460B439B0703D0A9
S3150800197009E008C9121F08C0042AFAD203E00B7846
S315080019800370401C491C521EF9D27047D2B201E0BE
S315080019900270401C491EFBD270470022F6E710B5BC
S315080019A013460A4604461946FFF7F0FF204610BDBF
S315080019B0F8B502464A40D40F42004B0052085B086D
S315080019C09A4202D20246084611464A0023D0C30D5F
S315080019D04A00DDB2120EAD1A202D35DA490201266B
S315080019E0490AF6058A19002C00D0524220214F1BBD
S315080019F01146B9402A411018C20D9A4221D0002C2E
S31508001A0017D0012D08DCDA05801AD20F8019D20703
S31508001A10DBB200F077FBF8BDDA05801A0123400037
S31508001A201B06C01880185A428018CA0F104349006E
S31508001A3007E04908C2071143DA05801A80194008E9
S31508001A40801800F057FBF8BD61000122511A001BEF
S31508001A50F7E70122D2075140AAE70122D2075040F0
S31508001A60A6E7024670B54A40D30FDB0740002DD0E3
S31508001A704A002AD0010E140E000212020919400A61
S31508001A80520A8418E50104465443000A120A2E0431
S31508001A905043A4194219200CC543AA18120C012553
S31508001AA0AD03521C521912047F39240400D0521C6B
S31508001AB0104301D44000491EC2B20C06C0092018C2
S31508001AC0401C4008802A02D003E0002070BD400870
S31508001AD04000002900DA0020184370BD70B50246A0
S31508001AE04A40D50F40004A00ED0740085208002832
S31508001AF014D0002A12D0C40DD30D41020120C0050E
S31508001B005202490A520AE41A091812187D349142F7
S31508001B1001D3641C00E04900002C01DA002070BDE6
S31508001B200023914201D3891A03434008490000283B
S31508001B30F7D100290AD0914202D10121C90705E04F
S31508001B40914201D2012101E00121C943E005C018F3
S31508001B50401900F0CFFA70BDF0B507460846584060
S31508001B6087B0C00F049048000E465900400849083F
S31508001B70BC1A884105D2384631461E4617460B46DA
S31508001B8002465800400810434CD0300D03904005DB
S31508001B905900400D490D0590401A0290402872DA06
S31508001BA018030121000B09050843019004980092C7
S31508001BB0002805D0019952420020884100920190E0
S31508001BC0029840210A1A0199009800F05FFA054622
S31508001BD00C466B4607CB00F07AFAC0197141039A96
S31508001BE00E0D0023D71756401A467A40164344D09E
S31508001BF0049A002A2DD0029A012A039A15DC1205A6
S31508001C00C01A914101263605001C7141D20F059E66
S31508001C10D2070093019202962A46234600F0B8FAA4
S31508001C2007B0F0BD38463146FAE71605224A0F4690
S31508001C30B218C01AB74101210905001C4F41001806
S31508001C407F41114618187941E20F10436D19644116
S31508001C5013E0E2076D0815436408C2071443039AA4
S31508001C6001261205C01A91413605001C7141CE079E
S31508001C70400830434908C01851412A46234600F017
S31508001C807AFACDE7FFE7049801224000C117121A35
S31508001C9000238B4104983146C417381AA141EEE750
S31508001CA030B40124E407634030BC55E730B401245E
S31508001CB0E407614030BC4FE70000E0FFF0B51FB411
S31508001CC088B00B990998002448400999C00F490023
S31508001CD049080991C0070B990090490049080B91DA
S31508001CE009990898A64608431CD00B990A980843F0
S31508001CF018D0099801244000420D4800410D099862
S31508001D0024050003000B204309900B980003000BE1
S31508001D1020430B9050181C49401800220190144685
S31508001D20104605E0002001460DB0F0BD032801DA93
S31508001D30034600E003239C46C11A0AAE0AE05F0088
S31508001D4008ADED5B4F00F75B7D430027AA187C4181
S31508001D50491C5B1E6145F2DD410004AB5A52210461
S31508001D60120C0A43240C401C0828DFDB0198029059
S31508001D700099704601910090059B049A0799069868
S31508001D8000F006FAD0E700000DFCFFFFF0B50C46A0
S31508001D905C4085B0E40FE40703944C000026640811
S31508001DA059009446490802460296224321D06246C3
S31508001DB00A431ED06200570D4A000E032303550D31
S31508001DC0012402462C492405781B1B0B360B4018A8
S31508001DD023432643614600901C46501AB44103D358
S31508001DE00098401C009002E0921800985B41002879
S31508001DF003DA0020014605B0F0BD002001210905DF
S31508001E000746864611E064461D46141BB54106D3AF
S31508001E106546521BB341744607430C43A646CD0795
S31508001E2040084908284392185B4105460D43EAD104
S31508001E301046184313D0604619465040714008436F
S31508001E4006D06046101AB34106D20122002306E0E6
S31508001E5000220123DB0702E00122D2435310009837
S31508001E6074460105381C6141029C039D00196941AD
S31508001E7000F081F9BFE70000FD030000C217C10F9B
S31508001E80504010B54018CA079623002100F03AF9C9
S31508001E9010BD10B500229623114600F033F910BD87
S31508001EA00EB5C217C10F5040CA0740180021054B8E
S31508001EB00293019200910A460B4600F069F903B0B5
S31508001EC000BD0000330400000EB50549029100214B
S31508001ED000910A460B46019100F05AF903B000BD7D
S31508001EE033040000C20F410040020123400ADB050B
S31508001EF0D207090EC0187F2901DA002070479629F3
S31508001F0003DC9623591AC84001E096398840002A0E
S31508001F10F4D040427047410040020122400AD205EF
S31508001F20090E80187F2901DA00207047962903DCFC
S31508001F309622511AC8407047963988407047000063
S31508001F404A0009030123090B1B051943094B10B560
S31508001F50520D9A4201DA002010BD064B34339A42DC
S31508001F6003DC9A1A00F0A2F810BD034951188840FC
S31508001F7010BD0000FF030000CDFBFFFFC20FD20714
S31508001F80400040080BD0C10D0723DB01C9184002E9
S31508001F900905400A1143C20840071143704700204B
S31508001FA00146704710B5002904DB0124E4074042C6
S31508001FB08C412146002B04DB1C460123DB075242D9
S31508001FC0A3418B4200D1824210BD0000CB0FDB0734
S31508001FD0490010B5490802460A4307D00A0D0724E6
S31508001FE00903E401090B121B002A01DC002010BDBD
S31508001FF0C900440F0C43C100E018D205801800F050
S3150800200079F810BD0122D207002800DB101A002932
S3150800201000DB511A814270470122D207002800DBF3
S31508002020101A002900DB511A88427047F0B51FB410
S315080020300646002082B005464024019100901BE028
S31508002040019922460F46304600F030F8049A059B5F
S31508002050801A994110D310461946224600F016F800
S31508002060361A8F410197224601200021009F00F071
S315080020700DF838184D4100902046641E0028DFDC14
S31508002080019B00982946324607B0F0BD10B5202AB4
S3150800209004DB0146203A9140002010BD91402023E0
S315080020A09C1A0346E3401943904010BD10B5202AF8
S315080020B004DB0846203AD040002110BD0B46D34029
S315080020C0D0402024A21A91400843194610BD10B5E5
S315080020D0202A06DBCB170846203A1041C1170B43C6
S315080020E006E00B461341D0402024A21A914008432B
S315080020F0194610BD002904DA401C490001D14008E0
S315080021004000704770B40024050C05D11024000463
S3150800211002D1002921D01124050E01D1000208346C
S31508002120050F01D10001241D850F01D18000A41CD3
S31508002130002801DB4000641C002908D020252E1B3E
S315080021400D46F540A14000D0012129430843010668
S315080021501B1B000ADB1D02D5002070BC7047DB057F
S31508002160181880180029F8DA401C4900F5D170BC07
S3150800217040084000704710B5002B08DA0024401CC0
S31508002180614192185B411A4301D14008400010BDD5
S31508002190F0B51FB482B005460C0003D0084602F01D
S315080021A001FE02E002F0FEFD2030024600902146C4
S315080021B02846FFF76BFF049B059A04460F4618430B
S315080021C01143084314D0184610431BD000984021E9
S315080021D00A1A18460599FFF769FF05460E46009A3A
S315080021E005990498FFF752FF084305D0012004E03B
S315080021F02046394607B0F0BD0020C11705430E43F7
S315080022002C43374300990E986305401A7905E40A6A
S3150800221000220C43FD0A0A3002D500200146E9E7F0
S315080022200105101969410C9C0D9D00196941FFF7BC
S31508002230A2FFDFE7FEB500231A461B1A8A4103DB15
S315080022400020014603B0F0BD4A000D0301212D0B05
S315080022500905520D0D43D10702D100186D41521ED2
S315080022605110FF31FF310131002704463E463846FA
S31508002270009701910246012100200905FFF716FF84
S31508002280C3197141F818324684468E464A4161465A
S315080022902846611A904104D36046241A9541764629
S315080022A01F46241900986D41401C00903428E1DD32
S315080022B0F91930467041091BA84103D20022D243BE
S315080022C0134601E00022134601980105381C7141A6
S315080022D0FFF751FFB6E70000064C0125064E05E05C
S315080022E0E36807CC2B430C3C98471034B442F7D329
S315080022F0FFF7ECFAA89B0008C89B000870B58C1875
S315080023000578401C6B075B0F01D10378401C2A1126
S3150800231006D10278401C03E006780E70401C491C62
S315080023205B1EF9D12B0705D40023521E0DD40B7062
S31508002330491CFAE70378401CCB1A921C03E01D7867
S315080023400D70491C5B1C521EF9D5A142D8D300203A
S3150800235070BD000010B50446002C08D101210920E3
S31508002360C00600F0E7FD002000F0E6F852E0012C78
S3150800237005D102210920C00600F0DCFD4AE0022C46
S3150800238005D104210920C00600F0D4FD42E0032C43
S3150800239005D108210920C00600F0CCFD3AE0042C3E
S315080023A005D110210920C00600F0C4FD32E0052C35
S315080023B005D120210920C00600F0BCFD2AE0062C24
S315080023C005D140210920C00600F0B4FD22E0072C03
S315080023D005D180210920C00600F0ACFD1AE0082CC2
S315080023E004D101210D4800F0A5FD13E0092C04D104
S315080023F002210A4800F09EFD0CE00B2C04D11021A6
S31508002400064800F097FD05E00C2C03D1802103480F
S3150800241000F090FD204600F08FF810BD000400483B
S315080024207FB500200090019002900390002427E0D9
S3150800243000250CE0E800294940186100405AA1002F
S315080024406A4651584018A1005050681C85B2142D90
S31508002450F0DBA1006A4650581421FFF75BFA2821E1
S31508002460484361001E4A515A3C225143461864218A
S315080024703046FFF74FFA6100194A5052601C84B281
S31508002480042CD5DB1748807E002826D014484088BF
S315080024901549884203DC1248808888420ADD1148BB
S315080024A02038C079002805D11049486005210D4813
S315080024B02038C1710A4840880A2803DB0848808802
S315080024C00A280ADA07482038C079002805D10749BA
S315080024D04860042103482038C1717FBDF4040020F8
S315080024E0740100202C040020E60F00000C020020D6
S315080024F000B587B001A800F0AFF80121480201F045
S31508002500F1F90020019070200290012080020390CA
S3150800251000200690059001A9064800F031F801212F
S31508002520044800F021F80121024800F011F807B02C
S3150800253000BD00000024014010B504460723002210
S315080025402146024800F038F810BD0000002401407A
S31508002550002904D0426801231A43426003E0426816
S315080025605208520042607047002904D08268082346
S315080025701A43826003E0826808239A4382607047A0
S3150800258042680B4B1A4042600B684A681A43436814
S315080025901A4342608268074B1A4082600B694A698F
S315080025A01A438B681A4383681A438260704700008F
S315080025B00FBCFFFF8FF1F9FFF0B504460D4616462E
S315080025C01F463F073F0F2B46082B0FD91B071B0F2C
S315080025D0083B606F9A000F21914088436067606FDF
S315080025E099003A468A40104360670BE0206F9A00CC
S315080025F00F21914088432067206F99003A468A4008
S3150800260010432067E0680121A9408843E060E0683C
S315080026100121A9400843E0600120800328400028E2
S3150800262003D0012000F020F807E00120C00328406D
S31508002630002802D0012000F017F8F0BD002905D0C7
S315080026408268FF2301331A43826004E08268FF230D
S3150800265001339A43826070470021016041608160BE
S315080026600173016141617047002806D0064949682F
S315080026700C221143044A516005E0034949680C22BB
S315080026809143014A516070470024014010B524481F
S315080026900078012834D10020214908702149088092
S315080026A012E02048008840001F49085A1F49098837
S315080026B0C9001F4A89181B4A1288520088521948AD
S315080026C00088401C17490880164800880428E8DB5B
S315080026D07E2002F0EDFA022000F02EF901211548BD
S315080026E0FFF7ACFF11480088401C104908800846CF
S315080026F00088142804DB0020088001200E49087091
S315080027000D480078002806D0FFF78AFE00200A49FF
S31508002710087000F059FC7E2002F0CAFA10BD0000CD
S31508002720840100209E010020BC040020A001002096
S31508002730F4040020002401407C010020FFB583B08A
S315080027400C46029400200190002726E000261CE093
S31508002750721C039951430846791CFFF7DBF80546B6
S31508002760A54201D9281B00E0601B05460298A8422D
S3150800277004D90295059806700698077002980028ED
S3150800278002D10120019002E0761C402EE0D300BF62
S315080027900198002800D002E07F1C042FD6D300BF82
S315080027A0029807B0F0BD000000BF00BF00BF00BF21
S315080027B000BFBFF34F8F00BF00BF00BF06480749E1
S315080027C0C86000BF00BF00BFBFF34F8F00BF00BF88
S315080027D000BF00BF00BFFDE70400FA0500ED00E0FA
S315080027E010B500F001F810BD10B523480078002890
S315080027F017D1224801F0FEF801283CD11F4800787D
S31508002800002838DD1D480078402834DC01F092FEA7
S315080028101B490860012018490870002019490870EA
S3150800282029E0164A17490978491C501801F0E2F8B8
S31508002830012816D113480078401C124908700F4821
S3150800284000780978884216D100200B4908700B4891
S315080028504078FF280FD10B48007802280BD1FFF7E4
S31508002860A3FF01F067FE064909686431884202D968
S3150800287000200149087010BD490100207804002095
S315080028804C0100204801002010B586B004460121FD
S31508002890880301F027F80121480401F003F8012212
S315080028A00921C80600F031FB01220A210920C006C9
S315080028B000F02BFB01A801F03EFF01943021684689
S315080028C0018100214181818101821821C18101A9EB
S315080028D0184801F0EDFE0121164801F0C6FE05A8CC
S315080028E000F069FB01214902684681820121817550
S315080028F01821C17505A90920C00600F0B9FA0121F9
S315080029008902684681824821C17505A90920C00641
S3150800291000F0AEFA1B2168460170032141700121BF
S31508002920817000F08BFF01220221024801F0B5FEFA
S3150800293006B010BD0038014001B506490098086088
S3150800294002E07E2002F0B4F9024800680028F8D1B7
S3150800295008BD000054010020014600220E4B1A61F2
S31508002960CA005A6100229A6105221A6100BF0A4A02
S315080029701069C207D20F002A04D0012212040240AD
S31508002980002AF4D0044A126952085200024B1A610E
S3150800299000229A617047000000E000E010B50021AF
S315080029A00448FFF74BFE022000F04AF801200249CE
S315080029B0087010BD002401408401002000B589B0CC
S315080029C00121084600F06EFF1A4800F045F801A8F4
S315080029D000F08EF8184801901848029000216846C1
S315080029E001730420049068460175802141754900E9
S315080029F0C182890001832021817609028183002111
S31508002A00C183018401A90B4800F04CF8012109484B
S31508002A1000F01CF801220221064800F039F80921C5
S31508002A2068460170022141700121817000F006FF9D
S31508002A3009B000BD0800024000240140BC04002083
S31508002A4001494860704700000000024002685208C9
S31508002A5052000A430260704710B5044620684008D1
S31508002A6040002060002020606060A060E060E1B265
S31508002A70084608380521FEF74DFF01460F20884015
S31508002A800249496808430149486010BD00000240F0
S31508002A90002A03D003680B43036002E003688B43F4
S31508002AA00360704710B50A7A8B7D1A430B7C1A436C
S31508002AB04B7C1A434B8A1A438B8A1A430B8B1A434D
S31508002AC04B8B1A430368094C23401A430260026879
S31508002AD00123DB039A438B8B1A430260CA68426060
S31508002AE00A6882604A68C26010BD00000F80FFFF56
S31508002AF00021016041600172C16001744174418224
S31508002B0081828175018341838183704770B506464A
S31508002B100C4621460A4800F04BF90546002D01D11E
S31508002B20401E70BD0648854202D10648051B00E0D6
S31508002B302D1B224629463046FEF716FF2046F0E7AB
S31508002B4000F4000800FC000870B506460C4621464D
S31508002B500A4800F02DF90546002D01D1401E70BD2A
S31508002B600648854202D10648051B00E02D1B224671
S31508002B7029463046FEF7F8FE2046F0E700F0000842
S31508002B8000F8000870B506460C4621460A4800F0CB
S31508002B900FF90546002D01D1401E70BD0648854235
S31508002BA002D10648051B00E02D1B22462946304661
S31508002BB0FEF7DAFE2046F0E700F8000800000108F4
S31508002BC070B505460C4622460249284600F0B1F87B
S31508002BD0204670BD00F4000870B505460C4622462E
S31508002BE00249284600F0A5F8204670BD00F0000806
S31508002BF010B50446084800690221084306490861D9
S31508002C0008464461006940210843034908610348AE
S31508002C1000F00EF910BD000000200240FF0F000072
S31508002C200C48C068C007C00F002801D001207047B3
S31508002C300848C06804210840002801D00220F6E7A9
S31508002C400448C06810210840002801D00320EEE798
S31508002C500420ECE70020024003480069802108436D
S31508002C6001490861704700000020024030B504465B
S31508002C700D46054800690121084303490861258076
S31508002C800F2000F0D5F830BD0020024010B57E2098
S31508002C9002F00EF8064800F00FF87E2002F008F859
S31508002CA0044800F009F87E2002F002F810BD000082
S31508002CB000F4000800F0000810B5044600F0ACF86F
S31508002CC02046FFF795FFFFF7C7FF10BD70B503460F
S31508002CD00125002208E050001C5A0748844201D00A
S31508002CE0002506E0501C82B2CE0F76187610964262
S31508002CF0F1DC00BF284670BDFFFF0000F8B50546A9
S31508002D000E46144600F088F87E2001F0D1FF002711
S31508002D1007E029883046FFF7A9FFB61CAD1C781CCA
S31508002D2087B2E10F09194910B942F2DCFFF794FF9F
S31508002D30F8BDF8B507460C4615462946204600F064
S31508002D4037F80646002E0DD12046FFF7B5FF0120BD
S31508002D5080022018FFF7B0FF2A4621463846FFF7BB
S31508002D60CDFF24E0012080022018401BB0420AD182
S31508002D70012080022018FFF79FFF2A463146384671
S31508002D80FFF7BCFF13E00120C0022018401BB04229
S31508002D9008D12046FFF790FF2A4631463846FFF706
S31508002DA0ADFF04E02A4631463846FFF7A7FFF8BDCF
S31508002DB0F8B505460E462F46E807C00F002801D08D
S31508002DC000BFFEE731460120C002FEF7B9FD002923
S31508002DD001D000BFFEE700240BE0204670434719E8
S31508002DE031463846FFF772FF012800D108E0601C1B
S31508002DF084B231460120C002FEF7A2FDA042ECDCF7
S31508002E0000BF31460120C002FEF79AFDA04200D15C
S31508002E1000273846F8BD00000248034948600348C1
S31508002E20486070472301674500200240AB89EFCD13
S31508002E3010B5024600BFFFF7F3FE0346521EFF24F5
S31508002E4000E0641E002CFCD1012B01D1002AF2D12E
S31508002E500648006977218843044908613420C86018
S31508002E60002A01D1052010BD1846FCE700200240C3
S31508002E70F8B50246CD782F073F0FCD781026354096
S31508002E80002D01D08D782F431446002011E08506C9
S31508002E902B0E0D88012686403540002D07D0256863
S31508002EA00F269E40B5433E469E4035432560451C49
S31508002EB0E8B20828EBDB141D0D882D1200950020BA
S31508002EC011E085062B0E01258540009E3540002D14
S31508002ED007D025680F269E40B5433E469E4035439B
S31508002EE02560451CE8B20828EBDBCD78282D04D1EF
S31508002EF055690E883543556106E0CD78482D03D1CE
S31508002F0015690E8835431561F8BD70B54D07EB0E8A
S31508002F10082902DA0546203501E0054624352C46FF
S31508002F200F269E402568B54316469E4035432560C4
S31508002F3070BD000038B504460D460920C006844217
S31508002F4003D10121480400F0ADFC1148844203D1A5
S31508002F500121000200F0A6FC0E48844203D101219B
S31508002F60000200F09FFC0C48844203D101210805A9
S31508002F7000F098FC684600F01EF8684605800121B6
S31508002F8081700021C17069462046FFF771FF38BD80
S31508002F900004004800080048000C004802469068F3
S31508002FA00840002801D0012070470020FCE7416155
S31508002FB07047016170470021C94301800221817071
S31508002FC00421C1707047000000B591B000200F9031
S31508002FD00E900D900C907E2001F06AFE0020109055
S31508002FE01FE010984000FE49085A0590FEF751FF69
S31508002FF0FC490690FEF772FD0790FEF7BFFF002218
S31508003000F94B09910890FEF759FE0B910A90FEF7C5
S31508003010DDFF10998900F54A50501098401C80B27F
S31508003020109010980428DCDBF0488068F049069078
S31508003030FEF754FD0790FEF7A1FFEE4AEE4B099105
S315080030400890FEF733FE0B910A90FEF7BFFF0F902C
S31508003050E6484068E6490690FEF740FD0790FEF709
S315080030608DFFE44AE44B09910890FEF71FFE0B9189
S315080030700A90FEF7ABFF0E900F98FEF77FFF00222F
S31508003080D94B05910490FEF711FE09910890DB488B
S315080030900F99FEF7E6FC0590FEF770FF079106907C
S315080030A0099B089AFEF772FE0B910A90FEF78EFFAF
S315080030B0D34908600E98FEF761FF0022CA4B0591B6
S315080030C00490FEF7F3FD09910890CC480E99FEF797
S315080030D0C8FC0590FEF752FF07910690099B089ACF
S315080030E0FEF754FE0B910A90FEF770FFC54908607B
S315080030F0C548008E322830DAC448408B0190FEF766
S31508003100E3FEC34AC34B03910290FEF7D7FD0022A4
S31508003110C14B05910490FEF739FE09910890BB480A
S31508003120408B0290FEF7B5FEBC490390FEF7D6FC2D
S315080031300490B34801680498FEF78FFC0590FEF7E3
S315080031401DFF07910690099B089AFEF71FFE0B9133
S315080031500A90FEF73BFF0D905CE0AB48008EBE2858
S315080031602CDAAA48408B0690FEF793FE0890A748EB
S31508003170808B0590FEF78DFEA9490690FEF7AEFCFA
S3150800318007900899FEF76DFCA4490990FEF7A6FC7E
S315080031900B909E48408B0790FEF77BFE9F49089050
S315080031A0FEF79CFC0990964801680998FEF755FCBD
S315080031B00A900B99FEF792FC0D902BE09348408BF2
S315080031C00690FEF766FE08909048008C0590FEF77C
S315080031D060FE93490690FEF781FC07900899FEF772
S315080031E040FC8E490990FEF779FC0B908748408B86
S315080031F00790FEF74EFE89490890FEF76FFC099086
S315080032007F4801680998FEF728FC0A900B99FEF793
S3150800321065FC0D907C48408E322830DA7B48008B5E
S315080032200190FEF751FE7A4A7A4B03910290FEF717
S3150800323045FD0022784B05910490FEF7A7FD0991FC
S3150800324008907248008B0290FEF723FE734903909C
S31508003250FEF744FC04906B4801680498FEF7FDFBF2
S315080032600590FEF78BFE07910690099B089AFEF7D4
S315080032708DFD0B910A90FEF7A9FE0C905CE0624862
S31508003280408EBE282CDA6148008B0690FEF701FEB8
S3150800329008905E48C08B0590FEF7FBFD60490690D6
S315080032A0FEF71CFC07900899FEF7DBFB5B490990C3
S315080032B0FEF714FC0B905548008B0790FEF7E9FDC6
S315080032C056490890FEF70AFC09904E480168099885
S315080032D0FEF7C3FB0A900B99FEF700FC0C902BE057
S315080032E04A48008B0690FEF7D4FD08904748408C64
S315080032F00590FEF7CEFD4A490690FEF7EFFB0790CC
S315080033000899FEF7AEFB45490990FEF7E7FB0B90D7
S315080033103E48008B0790FEF7BCFD40490890FEF733
S31508003320DDFB0990374801680998FEF796FB0A9075
S315080033300B99FEF7D3FB0C903A480D99FEF738FB2C
S315080033400B90FEF7E8FD3849086036480C99FEF7F9
S315080033502FFB0B90FEF7DFFD344908602A48008EE4
S31508003360314909684018C003010C27480186408E78
S315080033702E4909684018C003010C234841861B489A
S31508003380C0682B490A90FEF76CFB0B90FEF7C3FD4D
S3150800339081B21D48403001801C4870380088FF21E2
S315080033A0F531884276DD00201849703908800F48C3
S315080033B000680990FEF7E2FD1E4A1F4B0B910A9022
S315080033C0FEF7F0FD56D2094800680990FEF7D6FDCB
S315080033D01A4A1B4B0B910A90FEF7E4FD45D231E0E1
S315080033E07401002000F07F4500000840E404002036
S315080033F00000404125068195438BD43F0000484391
S315080034008C01002090010020CC0300207C020020C3
S31508003410091B9E5E29CB703F00408F4000007A440E
S31508003420002474490000C841940100209801002036
S315080034300000C842736891ED7C3FDD3F9CC420B014
S315080034407268D13F40212B48FFF7A8FD00280CD110
S3150800345029484079012808D12748C079002804D18D
S315080034602649486006212448C17101202249203195
S31508003470887314E02248006822490B90FEF7CCFDB9
S315080034800DD21D482030807E002804D11A492031EB
S31508003490887304E02CE00120174920318873184806
S315080034A0006819490B90FEF7B7FD04D201211248AE
S315080034B02030C17303E000210F482030C1730E4845
S315080034C02030807B00280ED10B484079012804D192
S315080034D001020848FFF76BFD0AE0FF2101310548A4
S315080034E0FFF767FD04E0FF2101310248FFF761FDA0
S315080034F011B000BD000400480C0400200C02002096
S31508003500E40400206F12233F333313400148806AD6
S3150800351070470000C0F7FF1F0148C06A70470000E7
S31508003520C0F7FF1F014800687047000058010020D7
S31508003530034800680349097840180149086070473C
S31508003540580100206001002008B50121480400F058
S31508003550A9F90121880400F0A5F96846FFF72BFDB3
S315080035600121C903684601804821C17069460920BE
S31508003570C006FFF77DFC6846FFF71DFD012109031C
S31508003580684601804821C17069460920C006FFF7D0
S315080035906FFC6846FFF70FFD40216846018004214D
S315080035A0C17069460148FFF763FC08BD000400487E
S315080035B010B50121C9030920C006FFF7EFFC002852
S315080035C069D17748807A00285AD175484079012808
S315080035D037D173482030807E002832D17148007870
S315080035E0401C704908700846007805281CDB002036
S315080035F0087004216C48FFF7DCFC6948903840895C
S31508003600002807D169486A4948600121644890380A
S31508003610418106E0002066494860002160489038EC
S31508003620418101F065FB0CE05E480078022808DC61
S315080036305F4840687D210901884202D900205C491B
S31508003640486057482030807E002816D15848406D7B
S315080036505849884211D3524890384089002805D1E4
S315080036605548534948650020486006E04D480078AB
S31508003670022802DC00204E49486001214848817230
S315080036804E48007800280DD101204C4908700121C8
S315080036904348817106E000204849087000214048E7
S315080036A0817181724248C0684049884272D90020B7
S315080036B03F49C86000213A4881712030807E002841
S315080036C062D108213848FFF774FC3548903840889D
S315080036D003285FDA32489038408900285AD13048A2
S315080036E04038408E5A280FDA2D482030C07B0028F3
S315080036F00AD12B48407901284CD1294920318876AE
S3150800370000202B49486045E025484079012802D128
S3150800371000202749486022484038408E5A282ADB2C
S31508003720274840882749884203DC254880888842FC
S3150800373008DD1B48C079002804D11D4948600521C9
S315080037401748C1711E4840880A2803DB1C48808830
S315080037500A2808DA1248C079002804D114494860B2
S3150800376004210F48C1710E48C079002812D10221E0
S315080037700B48C1710EE00A482030C07B012809D1E8
S3150800378001210748C17105E0002009494860002168
S31508003790034841717E2001F08BFA0148807910BDFB
S315080037A00C040020C400002000040048DC050000CA
S315080037B00C02002030750000606D0000A201002098
S315080037C074010020E60F000008B50121480400F046
S315080037D069F80121880400F065F86846FFF7EBFBF5
S315080037E0FF210E3168460180012181701021C170C8
S315080037F069461148FFF73CFBB6216846018001215E
S3150800380081701021C17069460920C006FFF730FB98
S3150800381010210920C006FFF7CAFB80210920C0062F
S31508003820FFF7C5FB01210448FFF7C1FB0821024841
S31508003830FFF7BFFB08BD0000000400488178002997
S3150800384025D017490322120289180278921092008D
S31508003850895802789207D30EFF229A4091434278FC
S315080038609207120E03789B07DB0E9A4011430C4A07
S3150800387003231B02D21803789B109B00D1500178B2
S31508003880CA06D20E01219140054A116007E0017867
S31508003890CA06D20E01219140014A80321160704752
S315080038A000E100E0002905D0054A52690243044BAD
S315080038B05A6104E0024A52698243014B5A617047D1
S315080038C000100240002905D0054AD2690243044B7C
S315080038D0DA6104E0024AD2698243014BDA61704731
S315080038E000100240002905D0054A92690243044B9C
S315080038F09A6104E0024A92698243014B9A617047D1
S315080039000010024010B500F031F804494968F02269
S3150800391011400909024A515CC84010BD0010024016
S315080039202201002010B5FFF7EDFF05494968072277
S3150800393012021140090A034A515CC84010BD000032
S31508003940001002402201002010B5FFF7DBFF0549F1
S3150800395049680722D2021140C90A034A515CC84085
S3150800396010BD00000010024022010020F8B51E48D4
S3150800397040680C210840042802D008282ED101E00E
S315080039801A4C2DE0184840300069C007C00F0028BF
S315080039900AD015484030006902210840002801D0A5
S315080039A0134802E0114800E0104807460E48403028
S315080039B00069FF2109040840000C451C0A484030EC
S315080039C00069072109020840000A461C394669436E
S315080039D008463146FDF79EFF044601E0034C00BF4A
S315080039E000BF2046F8BD00000010024000127A0011
S315080039F000093D0070B5044600250221074800F07D
S31508003A003AFE002808D0054800F08EFE20700221F4
S31508003A10024800F028FE0125284670BD00380140FE
S31508003A2010B500F001F810BD00B585B06248006811
S31508003A30012108436049086000BF5F480068022109
S31508003A4008400028F9D05D485D4908605D4800686F
S31508003A50102108435B49086008460068C008C00092
S31508003A60086057490968481E5749FDF753FF0490EF
S31508003A705448006804994907490F084351490860A2
S31508003A804D484068514908404B49486008464068D7
S31508003A9090210843484948600846406848604848B5
S31508003AA000684649884207D9434840680521090203
S31508003AB00843414948600BE0414800684449884248
S31508003AC006D93D4840680121890208433A494860B9
S31508003AD06B4601AA3A4801683E48FEF72FFE36486B
S31508003AE04030006980088000334940310861084643
S31508003AF00069400840000861684600784007400FA2
S31508003B000290684600794006400E03902A48C0692C
S31508003B10890508432849C8612748403000692E4965
S31508003B2008402549403108610398000402990902B2
S31508003B30084321494031096908431F494031086152
S31508003B401D4800680121090608431B49086000E072
S31508003B5000BF194800680121490608400028F7D027
S31508003B601548406880088000134948600846406840
S31508003B70022108431049486000E000BF0E4840682B
S31508003B800C2108400828F8D10120FEF7E5FE0A486E
S31508003B90406810218843084948600120FEF7DCFE8A
S31508003BA00548406880218843034948600120FEF79C
S31508003BB0D3FE05B000BD00000010024000A24A0472
S31508003BC0340100200020024000366E010FC0FFFFBE
S31508003BD00051250200127A00FFF800FF042806D1DA
S31508003BE00649096904221143044A116105E003499B
S31508003BF0096904229143014A1161704700E000E017
S31508003C0010B5FFF795FCA3480088401CA149088019
S31508003C1008464068401C48609F480088401C9E49EA
S31508003C2008809E480068002804D09C480068401E0A
S31508003C309A4908609A488079012805D19548C0684C
S31508003C40401C9449C86002E000209249C860944824
S31508003C502030407D012805D18E484069401C8D4999
S31508003C60486102E000208B4948618D48007A0128A6
S31508003C7005D18848006C401C8649086402E000208B
S31508003C8084490864834948680A21FDF743FE0029E8
S31508003C9027D183482030407A81492031097A8842E1
S31508003CA007DD7F482030007A401C7D4920310872A4
S31508003CB017E07B482030407A79492031097A8842D2
S31508003CC000D10EE076482030407A75492031097ACD
S31508003CD0884206DA72482030007A401E7049203140
S31508003CE008726F482030807E022804D06C48203045
S31508003CF0807E032804D16748806B401C6549886329
S31508003D0067482030C07A00280AD165482030807E6E
S31508003D10042805D15F48806C401C5E49886402E02F
S31508003D2000205C4988645E482030807E002803D1E4
S31508003D3058490865C86426E05948C07A012805D15B
S31508003D405448006D401C5349086502E0002051495B
S31508003D5008655348007B012812D14E48C06C401CA8
S31508003D604C49C8644E482030007B002804D10846D8
S31508003D708068401C886006E000204649886002E0AA
S31508003D8000204449C8644648807804280AD1414836
S31508003D90406D4449884208D23E48406D401C3D4922
S31508003DA0486502E000203B494865012109030920CE
S31508003DB0C006FFF7F3F8002813D039482030807B77
S31508003DC000280ED13648407901280AD13148806D3D
S31508003DD03549884208D22F48806D401C2D49886590
S31508003DE002E000202B4988652D482030007C0128F8
S31508003DF00AD12848C06D2D49884208D22548C06D89
S31508003E00401C2449C86502E000202249C8652448A8
S31508003E102030807C012805D11E48006E401C1D49B3
S31508003E20086602E000201B4908661D482030C07C51
S31508003E30012805D11748406E401C1649486602E01D
S31508003E400020144948667E2000F032FF40211848B9
S31508003E50FFF7A4F800280AD00E48C06E1549884214
S31508003E6008D20C48C06E401C0A49C86602E0002009
S31508003E700849C8660A482030007D012805D105484A
S31508003E80806E401C0349886602E000200149886666
S31508003E9010BD00000C020020500100205401002033
S31508003EA00C04002050C3000088130000701700009F
S31508003EB000040048B888000010B5164800680121BB
S31508003EC008431449086008464068134908401149E0
S31508003ED0486008460068114908400E4908600846C7
S31508003EE000680121890488430A4908600846406831
S31508003EF0C3210904884307494860084600680849F9
S31508003F000840044908609F2000048860FFF788FD80
S31508003F1010BD0000001002400CC0FFF8FFFFF6FEBF
S31508003F20FFFF8F0008B501214804FFF7BBFC0222FA
S31508003F3001210920C006FEF7E8FF02216846018034
S31508003F401821C1700121817069460920C006FEF753
S31508003F508FFF01214804FFF7A5FC0222114609201C
S31508003F60C006FEF7D2FF0421684601801821C170F9
S31508003F700121817069460920C006FEF779FF08BD50
S31508003F8030B587B004460D4601210846FFF79AFC6E
S31508003F9004A800F033F905946846058200210183D8
S31508003FA08176817404A90120800700F0F1F868463B
S31508003FB000F0D2F8602168460170012141700020A6
S31508003FC0019000216846017269460120800700F0C9
S31508003FD057F869460120800700F08AF80821C806C4
S31508003FE000F07EF80821C80600F0B0F8402108065F
S31508003FF000F038F84021080600F03CF8012188074F
S3150800400000F00AF80121880700F01EF80121880748
S3150800401000F00EF807B030BD002904D002688023EE
S315080040201A43026003E0026880239A4302607047DD
S31508004030002904D0026801231A43026003E00268DB
S315080040405208520002607047002905D0426C0123CD
S31508004050DB031A43426404E0426C0123DB039A4300
S3150800406042647047826907231B039A430B021A436B
S3150800407082617047C26970239A430A43C2617047D6
S3150800408010B5826907231B039A430B781B021A4350
S3150800409082610A7A12014B781B011A43036A30249B
S315080040A0A3431A4302624A6882630C4A904213D1B8
S315080040B04A7A12018B781B011A43036AC024A34368
S315080040C01A4302624A8992008B899B001A43436805
S315080040D02401A3431A43426010BD0000002C01408E
S315080040E082690123DB029A430B021A4382617047F5
S315080040F010B5C26970239A430B781A43C2610A7ACB
S3150800410012024B781B021A43036A03242402A343B0
S315080041101A4302624A68C2630B4A904213D14A7A2A
S3150800412012028B781B021A43036AA400A3431A439C
S3150800413002624A8912018B891B011A434368A4004B
S31508004140A3431A43426010BD002C0140C2690823EC
S315080041509A430A43C2617047002101704170817019
S315080041604160017241724181818170470122920743
S31508004170904201D1816301E08AB2826370470122CD
S315080041809207904201D1C16301E08AB2C2637047C7
S31508004190026803231B029A430B891A430260134AD7
S315080041A0904206D001229207904202D0104A9042CD
S315080041B005D1026870239A438B781A4302600B4A2A
S315080041C0904205D00B4A904202D00B4A904205D144
S315080041D0026B120A12028B7A1A4302634A68C26297
S315080041E00A8882620122426170470000002C014061
S315080041F00004004000440140004801400021C94332
S315080042004160002101800181817081727047000040
S3150800421010B50024BD48407D00280FD1BC48406831
S31508004220BC490968401ABC4988420BD90021B748DD
S31508004230203841710020B549887603E0B4484068C3
S31508004240B4490860B148407C002804D001287DD0D4
S3150800425002287CD139E1AD492039CA8CAC49486875
S31508004260C72105F099F80446A8482038408C9128BB
S3150800427005DA14220121002002F0EEF904E00022FA
S315080042800121104602F0E8F9A0482038C08CC82859
S3150800429009D09E482038C08CC72804D09B482038AF
S315080042A0C08CC92814D199486038408E9B49098822
S315080042B0884209D0002095490875C87408466038B0
S315080042C0408E9649088007E001209049C87403E0AB
S315080042D000208E490875C8748D48406E90498842FA
S315080042E047D98A482038408C401E8E49098888421A
S315080042F037DC86482038408C401C8A490988884221
S315080043002FDB82482038408CB42832DB7F4820389F
S31508004310818C408C814203D101207C49087509E0D3
S3150800432000207A4908757A498866486677482038A9
S31508004330418C81847648806E7949884219D902F081
S31508004340DBFE012071494874002001E01AE0D9E03B
S315080043506F49486674490870704908807149088031
S3150800436007E06A482038408C6E4908800020684972
S31508004370486600206D49087022460121084602F069
S315080043806BF9C0E0614920390A8C61494868C72140
S3150800439005F002F8044600220121084602F05CF9FD
S315080043A05A482038008CC82809D058482038008C2C
S315080043B0C72804D055482038008CC9281BD1534833
S315080043C06038008E55490988884210D000204F4928
S315080043D0087508462038408C5249088000204B4909
S315080043E0C87408466038008E4C49088007E00120EA
S315080043F04649C87403E0002044490875C8744B4808
S315080044000078002810D14249486640482038408C38
S31508004410AA2805DD00220121104602F01DF953E005
S315080044200120424908704FE03948406E3C498842AD
S3150800443045D936482038408C401E3A490988884272
S3150800444035DC32482038408C401C36490988884279
S315080044502DDB2E482038408CAA282DDB2B48203807
S31508004460408CB42828DA29482038818C408C81422F
S3150800447003D101202549087509E00020234908755C
S3150800448023498866486621482038418C818420481B
S31508004490806E234988420FD902201C49487402F0CD
S315080044A0C3FE00201A4948661F49087004E01748E9
S315080044B02038408C1B49088000201549486622464A
S315080044C00121002002F0C8F81DE011494868FF21C3
S315080044D0F531FDF71FFA002913D100200C4948666B
S315080044E0134948850122FE21572003F0B0FD00221A
S315080044F00121104602F0B0F800220121084602F018
S31508004500ABF800E000BF00BF10BD00002C0400207F
S315080045100C02002010010020C4090000160100202A
S31508004520DC0500000C010020F8000020180100201E
S315080045304804002010B5FEF7F5FF10BD70B5FFF76B
S31508004540E1F905467D21C900FDF7E4F90446601E38
S315080045500C49884200D90CE0601E0B4948610321CA
S31508004560081F00F045FC00200749886107200861FC
S3150800457000BF0420FFF732FB0021481E00F038FC7C
S3150800458070BD0000FFFFFF0000E000E010B502214B
S31508004590134800F079F8002820D0114800F0C4F834
S315080045A0C4B21048C078022811D10E4800790028F4
S315080045B010D10D488079AA2804D10B48C47101216D
S315080045C008480171AA2C05D10748847102E02046E3
S315080045D002F05AFF0221024800F045F810BD00001B
S315080045E0003801400C040020A405002010B504463C
S315080045F02146054800F09CF800BF0121024800F05A
S315080046003AF80028F9D010BD0038014070B50546C3
S315080046100E4600247E2000F04BFB00BF20E0042C51
S3150800462019DD701EA04216DD285D7E2806D17D2084
S31508004630FFF7DCFF5E20FFF7D9FF0FE0285D7D2836
S3150800464005D1FFF7D3FF5D20FFF7D0FF06E0285D11
S31508004650FFF7CCFF02E0285DFFF7C8FF601C84B2B5
S31508004660B442DCDB70BD4161704782695208520072
S315080046700A4382617047024690680840002801D0C4
S31508004680012070470020FCE70246D0680840002851
S3150800469001D0012070470020FCE7002A03D00369F7
S315080046A00B43036102E003698B4303617047000013
S315080046B070B504460D460026E069302188432979FD
S315080046C00843E061E06944218843A9790843E06129
S315080046D0E06980088000297A0843E061A06918210A
S315080046E0884369890843A061A06904218843297B16
S315080046F00843A0610B48844203D1FFF725F9064613
S3150800470002E0FFF70FF9064630462968FDF702F979
S315080047100009206230462968FDF7FCF80007000FFB
S31508004720606270BD0038014001464868C0B27047F3
S31508004730CAB2026070474B21C9010160302101717C
S31508004740002181710172182141810021017370478E
S3150800475010B51C484088030000F03BFB0504111EF9
S31508004760292A2B00174890300088FF211B318842E0
S3150800477004DA01211348418000F0BAFA19E0114819
S3150800478090300088FF210531884204DA02210D485D
S31508004790418000F0ADFA0CE00A4890300088F6280F
S315080047A004DA03210748418000F0A2FA01E000E09C
S315080047B000BF00BF034890304079002801D100F0BF
S315080047C097FA10BD7C03002010B57548408800286C
S315080047D006D0012845D0022871D0032840D199E097
S315080047E002216F489030817040216E48FEF7D6FB53
S315080047F0002827D06C494868FF21F531FDF78AF86B
S31508004800C007C00F00280ED180210920C006FEF778
S31508004810D0FB01216348FEF7CCFB10210920C00616
S31508004820FEF7C7FB1CE080210920C006FEF7BFFB88
S3150800483001215C48FEF7BBFB10210920C006FEF7E4
S31508004840B6FB0DE080210920C006FEF7B2FB012168
S315080048505448FEF7AEFB10210920C006FEF7A9FB57
S315080048609BE001214E489030817040214D48FEF76B
S3150800487095FB002813D04C494868FF21F531FDF710
S3150800488049F8C007C00F002804D101214548FEF7A2
S3150800489090FB08E001214348FEF789FB03E001216C
S315080048A04048FEF786FB80210920C006FEF77FFBFD
S315080048B010210920C006FEF77AFB6EE0FFE74021CB
S315080048C03848FEF76BFB002815D037494868FF21A2
S315080048D0F531FDF71FF8C007C00F002805D1802164
S315080048E00920C006FEF763FB0AE080210920C006FE
S315080048F0FEF75FFB04E080210920C006FEF759FB9E
S3150800490001212848FEF753FB10210920C006FEF7AF
S315080049104EFB42E040212348FEF740FB002815D015
S3150800492021494868FF21F531FCF7F4FFC007C00F9D
S31508004930002805D180210920C006FEF738FB22E0B1
S3150800494080210920C006FEF734FB1CE0164948689A
S31508004950CD21FCF7DFFFC007C00F002805D1802155
S315080049600920C006FEF723FB0DE00F494868CD2154
S31508004970FCF7D0FFC007C00F002804D0802109200B
S31508004980C006FEF716FB01210648FEF710FB1021AC
S315080049900920C006FEF70BFB00BF00BF10BD0000D4
S315080049A07C030020000400480C02002010B5A7482C
S315080049B08078030000F00DFA0504447DC0F0EF008E
S315080049C0A2480088FF211631884203DB01219F484F
S315080049D0817034E09D480088FF210C3188420ADD49
S315080049E09A4890384088022805D00221974890387E
S315080049F0418000F07DF940219548FEF7CFFA00285E
S31508004A001DD094494868FF21F531FCF783FFC0079C
S31508004A10C00F002805D180210920C006FEF7C7FA75
S31508004A2004E080210920C006FEF7C3FA10210920F8
S31508004A30C006FEF7BCFA01218548FEF7B8FA03E17D
S31508004A4082480088FF212731884203DB02217F48FC
S31508004A5081702DE040217E48FEF7A0FA002827D075
S31508004A607C494868FF21F531FCF754FFC007C00FA1
S31508004A70002804D101217648FEF799FA03E00121BE
S31508004A807348FEF796FA80210920C006FEF78FFACA
S31508004A9010210920C006FEF78AFA6C48903840882B
S31508004AA0012805D0012169489038418000F020F995
S31508004AB0CAE066480088FF212831884203DB0321C3
S31508004AC06248817037E040216148FEF767FA00289E
S31508004AD031D060494868FF21F531FCF71BFFC00754
S31508004AE0C00F00280ED180210920C006FEF761FA02
S31508004AF001215748FEF75DFA10210920C006FEF786
S31508004B0058FA0DE080210920C006FEF750FA102158
S31508004B100920C006FEF74BFA01214D48FEF747FA71
S31508004B204A4890384088002805D0002147489038E0
S31508004B30418000F0DDF887E040214548FEF72EFA6F
S31508004B40002843D0012109030920C006FEF726FAEA
S31508004B50002807D03F48806D3F49884202D9042182
S31508004B603A4881703B494868FF21F531FCF7D2FE87
S31508004B70C007C00F002810D180210920C006FEF703
S31508004B8018FA01213248FEF714FA10210920C00646
S31508004B90FEF70FFA0FE056E019E080210920C0065B
S31508004BA0FEF705FA10210920C006FEF700FA0121D2
S31508004BB02748FEF7FCF9254890384088002805D094
S31508004BC0002122489038418000F092F83CE04021CC
S31508004BD01F48FEF7E3F9002834D01C48903840886F
S31508004BE0002805D0002119489038418000F080F847
S31508004BF01848406D194988420ED280210920C006FE
S31508004C00FEF7D7F901211248FEF7D3F9102109203A
S31508004C10C006FEF7CEF90DE080210920C006FEF792
S31508004C20C6F910210920C006FEF7C1F90121084876
S31508004C30FEF7BDF905482030807B012802D1032103
S31508004C400248817000E000BF00BF10BD0C040020C0
S31508004C50000400480C020020941100003075000082
S31508004C600348806840084000014988607047000092
S31508004C70002C004080210143014A11607047000062
S31508004C80002C004003488068002801D001207047A6
S31508004C900020FCE7002C004010B5FFF7F3FF0028C2
S31508004CA004D0FFF7DDFF662000F002F810BD000013
S31508004CB04106490E014A116070470000002C004069
S31508004CC004494968FF22813291430143014A5160F0
S31508004CD070470000002C004004494968C909C90109
S31508004CE04206520E1143014A51607047002C00409B
S31508004CF010B57E20FFF7DCFF0948FDF7DDFF0949FF
S31508004D00094801860621303000F03DFA064930315F
S31508004D1088814022024904483030FEF70AF810BD5F
S31508004D2000F80008FBAA00004C03002070B50546F1
S31508004D300C460121C802FEF7C5FDFF208130FFF7AA
S31508004D40BFFF2046FFF7C8FF2846FFF793FF70BD51
S31508004D500FB410B503A9044B044A029800F09AF858
S31508004D6010BC08BC04B01847D5700008040200201F
S31508004D700FB41CB50246002007AC00290BD0491E0B
S31508004D8001910092064B6A462146069800F082F881
S31508004D90009A002111701CBC08BC04B0184700001A
S31508004DA0715100082021020C01D010211046020A78
S31508004DB001D010460839020901D01046091F820899
S31508004DC001D01046891E420801D0881E7047081A6D
S31508004DD0704730B47446641E2578641CAB4204D30D
S31508004DE0635D5B00E31830BC18471D46F8E7000012
S31508004DF010B5002819DB1A4A03231B02D2188308A8
S31508004E009B00D2588307DC0EFF23A3409A438B07E7
S31508004E101B0E8407E40EA3401A43114B03242402F5
S31508004E201B198408A4001A5118E00E4A03071B0F21
S31508004E30083B9B089B00D2588307DC0EFF23A34040
S31508004E409A438B071B0E8407E40EA3401A43054BAF
S31508004E500407240F083CA408A4001A5110BD00003A
S31508004E6000E100E01CED00E002E008C8121F08C1DE
S31508004E70002AFAD170477047002001E001C1121FCD
S31508004E80002AFBD1704700000149086070470000FE
S31508004E9008020020FFB58FB00F460446002606E03C
S31508004EA025280AD0129A11999047641C761C2078F6
S31508004EB00028F5D1304613B0F0BD00250121A14ADE
S31508004EC0009500E00543641C23780846203B98407B
S31508004ED01042F7D120782E2815D104200543607892
S31508004EE0641C2A280AD101CF641C00900BE00099A3
S31508004EF00A22514330394018641C00902078014634
S31508004F0030390929F3D920786C280ED004DC4C28CE
S31508004F1013D06A2812D104E074280ED07A280DD14D
S31508004F200BE001204005054307E0012109056278E9
S31508004F300D43824201D16D18641C641C2078864694
S31508004F4069284AD008DC0028B4D058286DD06328D0
S31508004F5010D0642808D140E070286BD0732812D08E
S31508004F60752860D0782860D0129A704611999047B3
S31508004F70761CE5E03878694608720020487202A86F
S31508004F800190012003E0386801900020C0433F1DCE
S31508004F9069070CD5002500E06D1C00998D420FDAD3
S31508004FA08542F9DB0199495D0029F5D108E000251C
S31508004FB000E06D1C8542FCDB0199495D0029F8D1AA
S31508004FC0761907E0019801990078491C0191129A0F
S31508004FD0119990476D1EF5D2B2E00A200290002181
S31508004FE06802400F039102280CD001CFC1178446EE
S31508004FF000290DDA6246084652420021814194464C
S315080050002D2008E0FF1DFF08FF0003CF8446EFE7C9
S31508005010280504D52B206A46107401203CE0E807D1
S315080050203AD02020F7E70A2000E01020002103915B
S31508005030029007E010200290002104200543082072
S31508005040039100906802400F022810D001CF00217A
S31508005050844600200D9028071FD5704670280CD06E
S31508005060029A1020039B42401A430CD015E0FF1DFC
S31508005070FF08FF0003CF8446EBE740206A4610741A
S3150800508001200D900CE06046084306D030206A46A1
S3150800509010747046507402200D907046582804D03B
S315080050A029A001900DA80E900DE02CA0F9E7604606
S315080050B0039B029AFCF7BAFF019B84469B5C0E9AF7
S315080050C0521E0E92137060460843F0D10E9805A939
S315080050D0081A20300190680701D5009801E00120E0
S315080050E000900199884203DD01460198081A00E0FC
S315080050F000200025009006E004A8129A405D119948
S3150800510090476D1C761C0D988542F5DB04E0129AD3
S31508005110302011999047761C0099481E0090002966
S31508005120F5DC08E00E980E990078491C0E91129A43
S3150800513011999047761C0199481E01900029F1DCC7
S31508005140641CB4E609280100303132333435363769
S3150800515038396162636465660000000030313233B5
S315080051603435363738394142434445460000000055
S315080051704A68002A06D00A68531C0B6010704868F3
S31508005180401E4860704710B502460023002901D129
S31508005190002010BD03E01488921CE01883B208466C
S315080051A04C1EA1B20028F6D11846F2E710B5BE4843
S315080051B04079002864D110210920C006FDF7F7FEC2
S315080051C080210920C006FDF7F2FE0121B748FDF748
S315080051D0EEFE0020B44920318876002301221946C4
S315080051E0184603F069F900231A461946184603F0CB
S315080051F063F9AF484068FF21F531884204D204219B
S31508005200AA48FDF7D6FE4DE10421A848FDF7CFFED2
S31508005210A7484068A7498842F5D9A348807A002854
S3150800522017D1A34840687D214901884201D2FFF77A
S315080052308FFA08219D48FDF7BAFE00219A48C171E8
S31508005240002099492031C872087399494862486311
S315080052500CE040219548FDF7A1FE002806D0002164
S31508005260914820308176012120384171202109207A
S31508005270C006FDF79CFE7D2040018D49486011E17E
S3150800528089482030807E0300FFF7A3FD060470B32B
S31508005290FEFDFC6F002084492031C87208738449DA
S315080052A048624863002301221946184603F004F9A8
S315080052B000231A461946184603F0FEF87A4840387D
S315080052C0418E01874030C078012808D17848406966
S315080052D07949884202D900217348C17010BD7448C3
S315080052E040687D210901884227D900207349087042
S315080052F06D48807A002802D16D49486002E07048FE
S315080053006B49486040216948FDF748FE00280CD1E2
S31508005310FFF71EFA08216548FDF749FE7E20FFF7CC
S31508005320C7FC1E20FDF708FB02E000206049486024
S3150800533004215E48FDF73BFE17E020210920C00640
S31508005340FDF737FE08215948FDF733FE58484068EF
S31508005350FF21F531884208D95348903840890028FA
S3150800536003D104215148FDF722FE9AE050484068CF
S31508005370FF21F531884204D204214C48FDF719FE75
S3150800538003E004214948FDF712FE4748C07805287E
S3150800539017D100220121084601F05EF9424840383B
S315080053A0018E4030C08B814205DA6422012100203B
S315080053B001F052F907E000220121104601F04CF9EC
S315080053C001E0FEF725FF38484038418E4030C08B53
S315080053D081420DDB34484038018E4030C08B814213
S315080053E006DB00203249486002202F4920318876A2
S315080053F057E02F484068FF21F531884204D204213E
S315080054002A48FDF7D6FD03E004212848FDF7CFFD1D
S31508005410274840682B4988421ED92348C08BD22882
S315080054201AD12148C08CCF2812DB1F48C08CD5283A
S315080054300EDA01201C49203188741D48006E1E4969
S31508005440884209D90122FE21672002F000FE03E006
S3150800545000201549203188741348C07805281AD1C8
S3150800546000220121084601F0F7F80F484038018E5E
S315080054704030C08B814208DA3C220121002001F02D
S31508005480EBF80AE00CE00AE008E0002201211046E9
S3150800549001F0E2F801E0FEF7BBFE02E001E000E001
S315080054A000BF00BF00BF19E70C0400200004004835
S315080054B00C020020B80B000088130000C40000206E
S315080054C0C40900001027000010B5BD48407900281F
S315080054D064D110210920C006FDF769FD8021092045
S315080054E0C006FDF764FD0121B648FDF760FD002002
S315080054F0B34920318876002301221946184602F05E
S31508005500DBFF00231A461946184602F0D5FFAE48B7
S315080055104068FF21F531884204D20421A948FDF7E5
S3150800552048FD4AE10421A748FDF741FDA648406821
S31508005530A6498842F5D9A248807A002817D1A248F8
S3150800554040687D214901884201D2FFF701F9082107
S315080055509C48FDF72CFD00219948C1710020984907
S315080055602031C87208739849486248630CE04021A4
S315080055709448FDF713FD002806D0002090492031F5
S31508005580887601218E48417120210920C006FDF741
S315080055900EFD7D2040018C4948600EE18848203088
S315080055A0807E0300FFF715FC060474B0FBFAF97356
S315080055B0002083492031C8720021814820300173B8
S315080055C0002081494862486300230122194618468B
S315080055D002F072FF00231A461946184602F06CFFBD
S315080055E077484038418E01874030C078012808D175
S315080055F0754840697649884202D900217048C170C9
S3150800560010BD714840687D210901884227D90020CC
S31508005610704908706A48807A002802D16A49486049
S3150800562002E06D486849486040216648FDF7B6FCC7
S3150800563000280CD1FFF78CF808216248FDF7B7FC63
S315080056407E20FFF735FB1E20FDF776F902E00020E5
S315080056505D49486004215B48FDF7A9FC17E0202155
S315080056600920C006FDF7A5FC08215648FDF7A1FC50
S3150800567055484068FF21F531884208D95048903886
S315080056804089002803D104214E48FDF790FC93E099
S315080056904D484068FF21F531884204D20421494823
S315080056A0FDF787FC03E004214648FDF780FC4448E3
S315080056B0C078062817D100220121104600F0CCFF39
S315080056C03F484038418E4030C08B814205DA50222F
S315080056D00121084600F0C0FF07E000220121084624
S315080056E000F0BAFF01E003F0A9FD35484038418EC5
S315080056F04030C08B814206DB0020334948600220D7
S315080057002F492031887657E02F484068FF21F53128
S31508005710884204D204212B48FDF74BFC03E0042100
S315080057202848FDF744FC284840682C4988421ED979
S315080057302348C08BD2281AD12148C08CCF2812DB27
S315080057401F48C08CD5280EDA01201D4920318874DF
S315080057501D48006E1E49884209D90122FE2167208C
S3150800576002F075FC03E000201549203188741448BE
S31508005770C07806281AD100220121104600F06CFFD5
S315080057800F484038418E4030C08B814208DA3C22AF
S315080057900121084600F060FF0AE00CE00AE008E094
S315080057A000220121084600F057FF01E003F046FDFC
S315080057B002E001E000E000BF00BF00BF20E70000F4
S315080057C00C040020000400480C020020B80B00005E
S315080057D088130000C4000020C40900001027000038
S315080057E010B56D484079002864D110210920C006FB
S315080057F0FDF7DDFB80210920C006FDF7D8FB012156
S315080058006648FDF7D4FB00216348203081760023E3
S3150800581001221946184602F04FFE00231A46194679
S31508005820184602F049FE5E484068FF21F531884275
S3150800583004D204215948FDF7BCFBABE004215748C4
S31508005840FDF7B5FB5648406856498842F5D952488F
S31508005850807A002817D1524840687D21490188423C
S3150800586001D2FEF775FF08214C48FDF7A0FB002181
S315080058704948C171002048492031C872087348490F
S31508005880486248630CE040214448FDF787FB00283E
S3150800589006D0002140482030817601212038417108
S315080058A020210920C006FDF782FB7D2040013C49E6
S315080058B048606FE038482030807E002804D00128F0
S315080058C065D0022865D163E0002133482030C172D3
S315080058D000203149203108733149486248632E480F
S315080058E04038418E01874030C078012808D12C48BD
S315080058F040692D49884202D900212748C17010BD48
S31508005900274840687D210901884227D90020274970
S3150800591008702148807A002802D12149486002E0AF
S3150800592023481F49486040211C48FDF737FB0028DB
S315080059300CD1FEF70DFF08211848FDF738FB7E202D
S31508005940FFF7B6F91E20FCF7F7FF02E0002014491E
S31508005950486004211148FDF72AFB17E02021092099
S31508005960C006FDF726FB08210C48FDF722FB0C486C
S315080059704068FF21F531884208D9074890384089A0
S31508005980002803D104210548FDF711FB01E000E0DA
S3150800599000BF00BF00BFB2E70C04002000040048A7
S315080059A00C020020B80B000088130000C400002079
S315080059B0C4090000F0B587B00020069005900024C1
S315080059C00025049000260027F748407D012814D1B9
S315080059D0F64840694B21C90088420ED90020F24991
S315080059E04875F2494861F2490880F2490870FF2172
S315080059F00131EF48801DFBF7D0FFEB4820380079CE
S31508005A0001286CD17E20FFF753F9E948C0790002D6
S31508005A10E749097A08430690E548407A0590E4483C
S31508005A20847AC67A0246117B507B01F081FE0746CE
S31508005A30DF4AD17A107B01F07BFE05460021DA4861
S31508005A40203801710121203041750020D74948616D
S31508005A50D94A0698811A904242D03CDCD74A811A24
S31508005A6090423ED01EDCD64A811A90423AD010DCCB
S31508005A70D44A811A904236D006DC442861D0D249ED
S31508005A804018002871D19CE201296FD00229F9D16A
S31508005A90D1E201296BD002296AD0032969D01029DD
S31508005AA0F0D151E32A297DD00CDC22297BD004DCF5
S31508005AB0012979D01129E5D1FAE3232975D02929B5
S31508005AC0E0D15DE0312971D0332970D044296FD0F7
S31508005AD05729D7D19CE0881E282846D204E0F2E34D
S31508005AE076E092E3C1E27AE243007B449B885B005E
S31508005AF09F446A00660072003B003B003B003B0087
S31508005B003B003B003B003B003B003B003B003B00AF
S31508005B103B003B0021020D024F022B027401850156
S31508005B20D5013B003B003B004000300148019C0189
S31508005B30BA013B003B009F00AB00F7001101C5000E
S31508005B40DF000598062809D1A048007800280BD15F
S31508005B5002F0A8FA01209D49087005E00598062874
S31508005B6002DD012002F09EFA12E2FDE34BE288E232
S31508005B709CE2C6E20022FE21E82002F068FAF3E77A
S31508005B808949203909880A2251430846FCF776F9DB
S31508005B908F490090FBF7A2FF8E490190FBF761FF42
S31508005BA0029006E0C7E39AE37CE3AEE318E0E1E39C
S31508005BB0EFE3FCF7B0F980B2039002F01CFAD3E7E2
S31508005BC0032002F06FFACFE7042002F06BFACBE766
S31508005BD0052002F067FAC7E7022002F063FAC3E776
S31508005BE0012C0AD171487030008B012300229721BD
S31508005BF00090FE2002F0CBF909E06C487030408B2B
S31508005C000223002297210090FE2002F0C0F9FAE351
S31508005C1004217148FDF7CDF9C820FCF78DFE042153
S31508005C206D48FDF7C4F90022FE21BD2002F00FFAE7
S31508005C30E9E35D48807E002806D05B486038028E1E
S31508005C40418E002002F034F9DDE3002C0AD15648D3
S31508005C506038408E00231A46F0210090FE2002F09C
S31508005C6096F90BE0012C09D14F486038008E0123C4
S31508005C700022F0210090FE2002F089F9C3E3002CEF
S31508005C800AD14A487030408800231A46F32100900A
S31508005C90FE2002F07CF90BE0012C09D14348703054
S31508005CA0808901230022F3210090FE2002F06FF97B
S31508005CB0A9E3002C03D13D487030458002E03B48FB
S31508005CC070308581394870308089FF21F5318842E6
S31508005CD006DA01F0DDF90022FE21F42002F0B7F918
S31508005CE091E3002C0AD131487030808800231A4687
S31508005CF0F1210090FE2002F04AF90BE0012C09D1AF
S31508005D002A487030C08901230022F1210090FE2024
S31508005D1002F03DF977E3002C03D1244870308580E2
S31508005D2004E0012C02D121487030C5811F4870302B
S31508005D308088FF21F53188420BDC1C487030C08909
S31508005D40884206DC01F0A4F90022FE21F22002F0C6
S31508005D507EF958E3002C0AD114487030C088002315
S31508005D601A46E9210090FE2002F011F909E0012CFB
S31508005D7007D1192001230022E9210090FE2002F014
S31508005D8006F940E3002C02D108487030C580FF2090
S31508005D902D30854206DA01F07BF90022FE21EA2041
S31508005DA002F055F92FE300002C0400200C02002015
S31508005DB0A4050020F1010020CBFE000066FE0000CD
S31508005DC055FE000052FE0000AF01FFFF0002002052
S31508005DD00000A0400000E04000040048002C0CD160
S31508005DE0FE4800896421484380B200231A46E2210E
S31508005DF00090FE2002F0CBF800E000BF03E3002C81
S31508005E0006D164212846FBF79BFD81B2F348018140
S31508005E10F2480089FF21F531884206DC01F038F99D
S31508005E200022FE21E32002F012F9ECE2002C0CD14C
S31508005E30EA4840896421484380B200231A46EB2188
S31508005E400090FE2002F0A3F80DE0012C0BD1E348E8
S31508005E50008A6421484380B201230022EB21009086
S31508005E60FE2002F094F8CEE2002C07D164212846E1
S31508005E70FBF766FD81B2D948418108E0012C06D1BD
S31508005E8064212846FBF75CFD81B2D448018201F003
S31508005E90FFF80022FE21EC2002F0D9F8B3E2012C2B
S31508005EA019D1CF48408803280BDACD484089002805
S31508005EB007D10121CA48B03081760020C749703918
S31508005EC048600022FE21E42002F0C1F80121C448FE
S31508005ED0903041711AE0002C13D10021C04890304F
S31508005EE041710020BE49B03188760022FE21E420A7
S31508005EF002F0ADF80020BB490870B849703948600F
S31508005F0004E00022FE21E42002F0A1F87BE2002C46
S31508005F100FD1B548C07A32280CDCB348C17AAF48ED
S31508005F20418201F0B5F80022FE21DF2002F08FF849
S31508005F3000E000BF67E2A948408A00231A46DE212E
S31508005F400090FE2002F023F85DE2002C0FD1A6484F
S31508005F50C07A32281CDCA448C17AA048818201F0A4
S31508005F6097F80022FE21E12002F071F810E0012CDA
S31508005F700ED19D48C07A32280ADC9B48C17A9748D8
S31508005F80C18201F085F80022FE21E12002F05FF8C7
S31508005F9039E2002C09D19148808A00231A46E0216B
S31508005FA00090FE2001F0F3FF0AE0012C08D18B488F
S31508005FB0C08A01230022E0210090FE2001F0E7FFBD
S31508005FC021E28A4985488183C1830184418401F09D
S31508005FD05FF80022FE21512002F039F813E2002C66
S31508005FE010D1002E03D17E48903007840AE0012E96
S31508005FF003D17B489030478404E0022E02D17848CA
S315080060009030C784FFE1002C14D1FDF77FFA049085
S315080060100498000C00231A4653210090FE2001F034
S31508006020B6FF049880B20123002253210090FE2077
S3150800603001F0ADFFE7E1002C0AD16848C08B00905B
S315080060406648838B00225421FE2001F066FF0BE090
S31508006050012C09D16148408C00906048038C0122CC
S315080060605421FE2001F059FFCDE1002C08D1012171
S315080060705B489030C170002202215D48FEF70DFB97
S31508006080C1E1002C11D1FF2101315748801DFBF7D2
S3150800609084FC002054490880022151489030C17080
S315080060A00022FE21562001F0D2FFACE1002C18D1C7
S315080060B000214B48B030417400204B490880032129
S315080060C047489030C1700121417120308176002007
S315080060D04249703948600022FE21572001F0B7FF77
S315080060E00EE0012C0CD100213D489030C1700020F3
S315080060F03B49B03188760122FE21572001F0A7FFDF
S3150800610081E1002C17D100203549B0314874364951
S315080061100880042132489030C17001214171203035
S31508006120817600202D49703948600022FE215820CA
S3150800613001F08DFF07E0012C05D100212848903099
S31508006140C170203081765EE1002C1AD100202649E4
S315080061500880062122489030C17001214171012032
S315080061601F49B031887600201C4970394860B4212F
S315080061701B489030C1830022FE21652001F067FF8D
S3150800618042E0012C18D1002017490880062114483E
S315080061909030C170012141712030817600200F496D
S315080061A070394860D2210E489030C1830022FE2102
S315080061B0652001F04CFF27E0022C25D100200A4972
S315080061C00880062106489030C170012141710120DE
S315080061D00349B0318876002000490BE07C02002094
S315080061E07C03002000020020A40500200410000003
S315080061F00038014070394860F0218448C183002284
S31508006200FE21652001F023FFFDE0002C17D10020B8
S315080062107F49088005217D48C1700121417101200F
S315080062207A492031887600207A494860B42177482F
S31508006230C1830022FE21662001F009FF30E0012C0F
S3150800624017D100207249088005217048C1700121C4
S31508006250417101206D492031887600206D494860DA
S31508006260D2216A48C1830022FE21662001F0EFFE92
S3150800627016E0022C14D100206549088005216348E0
S31508006280C170012141712030817600206149486042
S31508006290F0215E48C1830022FE21662001F0D7FE68
S315080062A0B1E005E000215948C17020308176AAE0A6
S315080062B0002C09D107215548C1700022FE217720FC
S315080062C001F0C5FE0AE09FE0012C07D100214F48E6
S315080062D0C1700122FE21772001F0B9FE93E0002C5F
S315080062E012D164220121002000F0B6F90022012112
S315080062F0084600F0B1F90120444920318876002289
S31508006300FE21882001F0A3FE7DE0002C12D1642234
S315080063100121084600F0A0F900220121104600F0EC
S315080063209BF901203949203188760022FE218920EF
S3150800633001F08DFE67E0384938480068FBF791FBA5
S315080063400190FBF7E8FD80B23349039034480068B2
S31508006350FBF787FB0190FBF7DEFD80B202900398FE
S3150800636000900022902100E04CE0FE20029B01F004
S31508006370D4FD48E0002C33D1002E0BD125487030CF
S31508006380C7830022FE21522001F061FE00F080FE44
S3150800639026E026E0012E0AD11E487030878300F0D9
S315080063A077FE0122FE21522001F051FE18E0022E4E
S315080063B00AD118487030478400F06AFE0222FE218E
S315080063C0522001F044FE0BE0032E09D1114870302B
S315080063D0078400F05DFE0322FE21522001F037FEFD
S315080063E011E0002C0DD101200849203188760121C1
S315080063F00648417101200549203188750020054964
S31508006400486000E000BF00BF07B0F0BD0C040020E4
S31508006410A40500200C02002000007A449001002008
S315080064208C010020F0B589B00020089007900690EE
S315080064305048007901287DD14F488079AA287AD119
S315080064404D48C079322877DA4B48C079002873DD81
S315080064504949C97908461938FBF710FD0890089884
S31508006460FBF78CFD0646454A454BFBF727FC0446D9
S315080064700022444BFBF770FB0391029042480068E8
S31508006480FBF77CFD01910090039B029AFBF77EFCCB
S3150800649005910490FBF79AFD07900898FBF76EFDA7
S315080064A00446364A364BFBF709FC0022354B019168
S315080064B00090FBF751FB0391029034480068FBF704
S315080064C05DFD0646039B029AFBF760FC0591049066
S315080064D0FBF77CFD06902E490798FBF793FD38D20B
S315080064E02C490798FBF798FD33D229490698FBF7FC
S315080064F089FD2ED227490698FBF78EFD29D2264913
S315080065000798FBF7AEFA0446FBF705FD81B2234868
S31508006510418321490698FBF7A4FA0446FBF7FBFCDE
S3150800652081B21E48018300F0B3FD1C48408B0090E1
S315080065301A4802E01BE017E013E0038B00226021F3
S31508006540FE2001F0EAFC0122FE21562001F07FFD23
S3150800655004E00222FE21562001F079FD00210548BB
S31508006560C17000210348C17000210248017109B0B9
S31508006570F0BD00000C040020A4050020091B9E5E47
S3150800658029CB703F0000F03F8C01002090010020CD
S31508006590000018410000E04000007A447C02002018
S315080065A029494A88498A511A814209DB264970399C
S315080065B08968254A703AD1620021244A11701AE086
S315080065C021494988814216DC20490978002912D1D7
S315080065D01F490A880A8301211C4A11701A49703911
S315080065E08968194A703AD26A891A174A703A516202
S315080065F011468968516314498A88898A511A8142E1
S3150800660009DB0021134A11700F49703989680E4A4F
S31508006610703A116317E00C498988814213DC0D49E9
S31508006620097800290FD10A490A884A830121094AAB
S315080066301170054970398968034A703A126B891ACC
S31508006640014A703A916270477C020020E4000020FB
S315080066500C040020E500002070B505460E461446D9
S31508006660002E02D0012E4AD120E0002D02D0012DA5
S315080066701AD10CE0602101208007FDF7F3FC002108
S3150800668001208007FDF772FD1E4804700CE06021AA
S3150800669001208007FDF7EEFC002101208007FDF7A9
S315080066A06EFD1948047000BF00BF28E0002D02D017
S315080066B0012D22D110E013480078A0420BD06021AA
S315080066C001208007FDF7CEFC214601208007FDF753
S315080066D04DFD0C48047010E00B480078A0420BD022
S315080066E0602101208007FDF7C5FC214601208007AF
S315080066F0FDF745FD0448047000BF00BF00BF00BF9A
S3150800670070BD0000A3010020A401002010B5F348C5
S315080067104079012879D1F1482030007E0028F9D146
S31508006720EE48C0790300FEF754FB0805075DB0FD87
S31508006730FCFBFAF9002010BDE9494868FF219131B0
S31508006740FBF7E8F88007800F002809D18021092087
S31508006750C006FCF72CFC0121E248FCF728FC3AE0CD
S31508006760DF494868FF219131FBF7D4F88007800F8D
S31508006770012809D180210920C006FCF71AFC01214D
S31508006780D848FCF714FC26E0D5494868FF21913122
S31508006790FBF7C0F88007800F022809D1802109205D
S315080067A0C006FCF704FC0121CE48FCF700FC12E009
S315080067B0CB494868FF219131FBF7ACF88007800F79
S315080067C0032808D10121C748FCF7F3FB80210920DB
S315080067D0C006FCF7ECFB10210920C006FCF7E7FB16
S315080067E00120A8E7BE494868C821FBF793F8800747
S315080067F0800F00280AD180210920C006FCF7D7FBA4
S315080068000121B848FCF7D3FB38E065E1B44948688C
S31508006810C821FBF77FF88007800F012809D180215E
S315080068200920C006FCF7C5FB0121AE48FCF7BFFBF3
S3150800683024E0AB494868C821FBF76CF88007800F4D
S31508006840022809D180210920C006FCF7B0FB0121E6
S31508006850A448FCF7ACFB11E0A1494868C821FBF73E
S3150800686059F88007800F032808D101219D48FCF7B5
S31508006870A0FB80210920C006FCF799FB10210920FE
S31508006880C006FCF794FB012055E795494868C821DE
S31508006890FBF740F88007800F002809D180210920DE
S315080068A0C006FCF784FB01218E48FCF780FB3DE01F
S315080068B08B494868C821FBF72DF88007800F012807
S315080068C009D180210920C006FCF773FB0121854800
S315080068D0FCF76DFB2AE082494868C821FBF71AF8DD
S315080068E08007800F022809D180210920C006FCF7FD
S315080068F05EFB01217B48FCF75AFB17E0784948689C
S31508006900C821FBF707F88007800F03280ED101215D
S315080069107448FCF74EFB8021092004E0DBE0B2E076
S315080069205FE034E009E0C006FCF741FB10210920CE
S31508006930C006FCF73CFB0120FDE669494868FF21D3
S315080069402D31FAF7E7FFC007C00F002805D18021CF
S315080069500920C006FCF72BFB0EE061494868FF21B9
S315080069602D31FAF7D7FFC007C00F002804D08021C1
S315080069700920C006FCF71DFB10210920C006FCF7FC
S3150800698016FB01215748FCF712FB0120D3E65449B0
S315080069904868FF219131FAF7BDFFC007C00F0028EC
S315080069A005D180210920C006FCF701FB0EE04C4901
S315080069B04868FF219131FAF7ADFFC007C00F0028DC
S315080069C004D080210920C006FCF7F3FA102109201B
S315080069D0C006FCF7ECFA01214248FCF7E8FA012068
S315080069E0A9E63F494868C821FAF794FF8007800F4F
S315080069F0002809D180210920C006FCF7D8FA012110
S31508006A003848FCF7D4FA37E035494868C821FAF718
S31508006A1081FF8007800F012809D180210920C0063F
S31508006A20FCF7C7FA01212F48FCF7C1FA24E02C49E4
S31508006A304868C821FAF76EFF8007800F022809D137
S31508006A4080210920C006FCF7B2FA01212548FCF787
S31508006A50AEFA11E022494868C821FAF75BFF8007B9
S31508006A60800F032808D101211E48FCF7A2FA8021CD
S31508006A700920C006FCF79BFA10210920C006FCF77E
S31508006A8096FA012057E616494868C821FAF742FFE0
S31508006A90C007C00F002805D180210920C006FCF7D1
S31508006AA086FA0DE00E494868C821FAF733FFC00791
S31508006AB0C00F002804D080210920C006FCF779FA07
S31508006AC010210920C006FCF772FA01210548FCF7D7
S31508006AD06EFA01202FE600BF00BF2CE60C0400204A
S31508006AE00C0200200004004810B5FE48807E0028ED
S31508006AF074D0FC486038408EFF217D31884204DC22
S31508006B00F8486038008E88421CDDF6482038C0797F
S31508006B10002817D1F44840880A2813DDF24840882F
S31508006B20F24988420EDAF04880880A280ADDEE48DB
S31508006B308088884206DA0020ED4948600321E94842
S31508006B402038C171EA48006CEA4988420AD9E54802
S31508006B502038C079002805D1E54948600321E14875
S31508006B602038C171DF48807E042838D1DD48C07AD4
S31508006B7000282BD1DB482038C07A01281ED1DC48F2
S31508006B80006DDD49884231D90020D9490865D548C4
S31508006B906038C18E008E81420BDBD2482038C0791E
S31508006BA0002823D1D24948600721CE482038C17130
S31508006BB01CE0CC486038018EC18617E00020CC491D
S31508006BC00865C8486038018EC1860FE00020C849AC
S31508006BD00865C4486038018EC18607E028E00020B1
S31508006BE0C3490865BF486038018EC186BD48807EA6
S31508006BF001282BD1BB482038007B01281ED1BC4870
S31508006C00C06CBD49884228D90020B949C864B5482E
S31508006C106038818E408E81420BDBB2482038C079BD
S31508006C2000281AD1B24948600721AE482038C171F8
S31508006C3013E0AC486038418E81860EE00020AC49EE
S31508006C40C864A8486038418E818606E00020A849B5
S31508006C50C864A4486038418E8186A24820384079A5
S31508006C60012877D19F482038C07900280BD0002307
S31508006C7001221946184601F01FFC00231A46194638
S31508006C80184601F019FC97482038C0790300FEF72A
S31508006C90A0F80805073C71A4D8FDFCFB002010BD30
S31508006CA093484068E121C900884229D91021092062
S31508006CB0C006FCF77CF980210920C006FCF777F9A5
S31508006CC001218E48FCF773F90120864908760846A3
S31508006CD0807D002807D186494860002181482038F0
S31508006CE04171C17108E082484068AF2109018842B4
S31508006CF002D900207E49486001207A49C87502E019
S31508006D000020784908760120C9E7794840687C4917
S31508006D1088422AD910210920C006FCF748F98021A3
S31508006D200920C006FCF743F901217448FCF73FF92E
S31508006D3001206C4908760846807D00280BD16C49ED
S31508006D4048600021674820384171C17100206849B0
S31508006D5048600DE02BE166484068AF21090188428A
S31508006D6006D900206249486002E000205D4908769D
S31508006D70012094E75E4840686249884228D9102174
S31508006D800920C006FCF713F980210920C006FCF784
S31508006D900EF901215948FCF70AF9012051490876EC
S31508006DA00846807D00280AD15149486000214D488F
S31508006DB020384171C17100204D4948600BE04C48AC
S31508006DC040685149884206D900204949486002E08E
S31508006DD0002044490876012061E7454840687D213E
S31508006DE00901884228D910210920C006FCF7DFF8D6
S31508006DF080210920C006FCF7DAF801213F48FCF794
S31508006E00D6F80120374908760846807D00280AD139
S31508006E10374948600021334820384171C171002044
S31508006E20334948600BE0324840683349884206D9FE
S31508006E3000202F49486002E000202A4908760120F0
S31508006E402DE72B484068E121C90088422DD9102139
S31508006E500920C006FCF7ABF880210920C006FCF71C
S31508006E60A6F801212548FCF7A2F801201D49087655
S31508006E700846807D00280ED11D4948600021194822
S31508006E8020384171C17102E090E05CE012E0002018
S31508006E90174948600CE016484068AF210901884246
S31508006EA006D900201249486002E000200D490876FC
S31508006EB00120F4E60E4840681349C83988423CD98F
S31508006EC010210920C006FCF772F880210920C006A7
S31508006ED0FCF76DF801210948FCF769F8012001491A
S31508006EE0087613E02C04002074010020E60F000049
S31508006EF00C02002070110100B80B000000040048C5
S31508006F00A4060000C4090000AC0D00000846807DF8
S31508006F10002809D127494860002127484171C171D5
S31508006F200020244948600CE02248406823498842EA
S31508006F3007D900201F49486003E000211E48203079
S31508006F4001760120ABE61B4840681D49884227D9CF
S31508006F5010210920C006FCF72AF880210920C0065E
S31508006F60FCF725F801211748FCF721F801211248FA
S31508006F7020300176807D002809D10E49486000211D
S31508006F800D484171C17100200A4948600CE0094862
S31508006F9040680D49884207D900200649486003E041
S31508006FA00020054920310876012078E600BF00BF99
S31508006FB075E600000C0200200C040020CC1000002E
S31508006FC0A4060000000400488C0A000010B5052439
S31508006FD021E080212C48FAF7E0FC80212A48FBF7BB
S31508006FE095FD12212848FEF7CEF82749898C884254
S31508006FF00CD125483038008E2449884204D000F048
S3150800700051FC00F045F800E010BD04E0002000E067
S31508007010401C8028FCDB2046611ECCB20028D8D153
S3150800702000BF052423E080211748FAF7B6FC802123
S315080070301548FBF789FD12211348FEF7A4F81249F3
S31508007040898C88420ED110483038008E0F49884204
S3150800705004D000F027FC00F01BF802E000F018F856
S31508007060D2E704E0002000E0401C8028FCDB204634
S31508007070611ECCB20028D6D100BF00F013FC00F088
S3150800708007F800BFC0E700007C020020FBAA00004A
S3150800709010B57E20FDF70CFEFBF7F8FD0B490C48F2
S315080070A0018612213030FEF76EF80949303188849E
S315080070B0802107483030FBF783FD7E20FDF7F8FD79
S315080070C0802103483030FBF787FD10BDFBAA00007E
S315080070D04C02002070B504460D46E1B20548FDF79E
S315080070E027FB00BF01210348FDF7C5FA0028F9D0A0
S315080070F0204670BD00380140F0B587B00024002056
S31508007100069005904049088BFAF7C3FE07463F49A3
S31508007110FAF7E4FC05463C49088BFAF7BAFE3B4900
S315080071200490FAF7DBFC0746394801683846FAF74F
S3150800713094FC06462946FAF7D1FC06903549C88CD0
S31508007140FAF7A7FE06463449FAF783FC05462946A8
S315080071500698FAF7C3FC059030490598FAF781FCBA
S315080071600546FAF7D8FE81B22748C183C08B00903E
S315080071702548838B00225421FE2000F0CEFE2249AA
S31508007180088BFAF786FE20490190C88BFAF781FE2C
S3150800719022490090FAF7A2FC07460199FAF761FC22
S315080071A006461A49FAF79AFC17490390088BFAF724
S315080071B070FE07461549FAF791FC06461448016819
S315080071C03046FAF74AFC02900399FAF787FC054617
S315080071D01149FAF7EDFB0490FAF79DFE84B20A48C6
S315080071E0C08B0F49884204DB0748C08B0D4988428B
S315080071F004DD0222FE21572000F029FF0548403809
S315080072004486204607B0F0BD7C02002000007A4480
S31508007210900100200C0400200000C8410024744995
S31508007220B80B000088130000F0B587B000240020D2
S31508007230069005904049488BFAF72BFE07463F49CA
S31508007240FAF74CFC05463C49488BFAF722FE3B49BF
S315080072500490FAF743FC0746394801683846FAF7B6
S31508007260FCFB06462946FAF739FC06903549088C90
S31508007270FAF70FFE06463449FAF7EBFB05462946A8
S315080072800698FAF72BFC059030490598FAF7E9FBBA
S315080072900546FAF740FE81B227488183C08B0090E5
S315080072A02548838B00225421FE2000F036FE224911
S315080072B0488BFAF7EEFD20490190C88BFAF7E9FDED
S315080072C022490090FAF70AFC07460199FAF7C9FB22
S315080072D006461A49FAF702FC17490390488BFAF74B
S315080072E0D8FD07461549FAF7F9FB0646144801681A
S315080072F03046FAF7B2FB02900399FAF7EFFB054618
S315080073001149FAF755FB0490FAF705FE84B20D48C1
S31508007310403804860848808B0D49884204DB0648B5
S31508007320808B0C49884204DD0222FE21572000F09A
S315080073308EFE204607B0F0BD7C02002000007A448D
S315080073408C0100200C0400200000C8410024744968
S31508007350B80B000088130000F0B587B000240020A1
S31508007360069005904049488BFAF793FD07463F4932
S31508007370FAF7B4FB05463C49488BFAF78AFD3B49C0
S315080073800490FAF7ABFB0746394801683846FAF71E
S3150800739064FB06462946FAF7A1FB06903549088C90
S315080073A0FAF777FD06463449FAF753FB05462946A8
S315080073B00698FAF793FB059030490598FAF751FBBA
S315080073C00546FAF7A8FD81B227480184408C00904B
S315080073D02548038C01225421FE2000F09EFD2249F7
S315080073E0488BFAF756FD20490190088CFAF751FDAB
S315080073F022490090FAF772FB07460199FAF731FB22
S3150800740006461A49FAF76AFB17490390488BFAF7B2
S3150800741040FD07461549FAF761FB06461448016818
S315080074203046FAF71AFB02900399FAF757FB054616
S315080074301149FAF7BDFA0490FAF76DFD84B20A48C5
S31508007440008C0F49884204DB0748008C0D498842A6
S3150800745004DD0222FE21572000F0F9FD05484038D8
S315080074600486204607B0F0BD7C02002000007A445E
S315080074708C0100200C0400200000C8410024744937
S31508007480B80B00008813000070B5044600257E205E
S31508007490FDF70EFCA348008840280ADD0020A14914
S315080074A00880A1490870FF2101319E48801DFAF71E
S315080074B074FA9D4800780300FDF78BFC0805213611
S315080074C04760DAF1F0EF0020964948717E2C0FD11B
S315080074D00880012094490870924801880088401C59
S315080074E0904A1080901D445400201146C87002E04E
S315080074F000208C49088000208A4908710FE1FE2C7B
S3150800750001D0002C0FD1874801880088401C854A85
S315080075101080901D44540220834908701046007953
S31508007520001911460871FAE07E4801880088401C57
S315080075307C4A1080901D445403207B4908701046ED
S315080075400079001911460871E9E076480188008833
S31508007550401C744A1080901D4454042072490870D7
S31508007560104600790019114608710846C470C0789B
S31508007570002802D105206C490870D0E06948407996
S31508007580012856D15E2C1CD1664800797E306549A3
S3150800759008717E21634802880088401C614B188068
S315080075A0981D8154801FC078401EC0B21946C87005
S315080075B0002802DC05205C490870002059494871FA
S315080075C055E05D2C1CD1574800797D305549087126
S315080075D07D21544802880088401C524B1880981D0B
S315080075E08154801FC078401EC0B21946C870002852
S315080075F002DC05204C49087000204A49487136E0EB
S3150800760048480079001947490871084601880088E2
S31508007610401C444A1080901D4454801FC078401E68
S31508007620C0B21146C870002821DC05203E49087002
S315080076301DE07D2C03D101203A49487117E03948ED
S315080076400079001937490871084601880088401CE6
S31508007650344A1080901D4454801FC078401EC0B222
S315080076601146C870002802DC05202F49087056E02C
S315080076702C480079C043401CC5B27D2D05D15D2C30
S3150800768017D106202849087013E07E2D08D15E2CF4
S315080076900FD10620244908700BE03FE02FE011E0E7
S315080076A0A54203D106202049087002E007201E499A
S315080076B008701C4801880088401C1A4A1080901DD2
S315080076C044542CE0174801880088401C154A10804D
S315080076D0901D44547E2C08D10121144801710020C4
S315080076E0114608801049087008E000200D490880F6
S315080076F000210E48017100200B4908700FE0002098
S3150800770009490870074801880088401C054A108006
S31508007710901D445400201146088000E000BF00BFB9
S3150800772070BD0000A4050020F10100200C04002013
S3150800773070B50246002013460C461D02FF26360287
S3150800774035402543284670BD86B004460D46266852
S315080077506768A0680590E0680490206903906069EE
S315080077600290A0690190E069009017A0FDF7F0FA71
S3150800777031461BA0FDF7ECFA39461CA0FDF7E8FADE
S315080077801DA00599FDF7E4FA1EA00499FDF7E0FA95
S315080077901FA00399FDF7DCFA20A00299FDF7D8FA95
S315080077A023A00199FDF7D4FA26A00099FDF7D0FA8F
S315080077B02948416A29A0FDF7CBFA29462BA0FDF7EF
S315080077C0C7FA00BFFEE700005B4861726420666185
S315080077D0756C742068616E646C65725D0D0A0000D4
S315080077E05230203D2025780D0A0000005231203DF8
S315080077F02025780D0A0000005232203D2025780DFC
S315080078000A0000005233203D2025780D0A000000AA
S31508007810523132203D2025780D0A000053746163E9
S315080078206B6564204C52203D2025780D0A00000027
S31508007830537461636B6564205043203D2025780DA1
S315080078400A000000537461636B656420505352202C
S315080078503D2025780D0A000000ED00E05343425F05
S3150800786053484353523D25780D0A000043757272FA
S31508007870656E74204C52203D2025780D0A000000C4
S315080078800649074801860021303041805F21818002
S31508007890C18001810021418170470000FBAA0000D8
S315080078A04C03002000B5154915480186FF210F3104
S315080078B0303041800A210181A021C180C821818000
S315080078C078214181B221C18132210182BE21818183
S315080078D00C4901830B4925394183052141820A2137
S315080078E08182C18208498183C1830184418412212E
S315080078F0FDF749FC02493031888400BDFBAA000027
S315080079004C020020782100000410000010B57E20EB
S31508007910FDF7CEF9FEF7FAFE012800D110BD604842
S31508007920407901287ED15E482030807E002802D02A
S31508007930012860D137E040215A48FBF72FFB002881
S315080079401DD157482030407E012805D100205649D0
S3150800795048605349203148765348406D5349884218
S3150800796020D2514840687D21090188421AD24C48E4
S3150800797090384089002815D1FCF726FF12E04848C0
S315080079802030407E002803D1012045492031487621
S315080079904548C06E4549884202D2FCF715FF01E00A
S315080079A0FDF704F879E040494868FF21F531F9F711
S315080079B0B1FFC007C00F00280ED180210920C006DC
S315080079C0FBF7F7FA01213748FBF7F3FA10210920EC
S315080079D0C006FBF7EEFA0DE080210920C006FBF78A
S315080079E0E6FA10210920C006FBF7E1FA01212D4825
S315080079F0FBF7DDFA51E02A482030807E052829D198
S31508007A0029494868FF21F531F9F784FFC007C00FF7
S31508007A10002810D180210920C006FBF7CAFA0121E7
S31508007A20204800E03AE0FBF7C4FA10210920C00616
S31508007A30FBF7BFFA30E080210920C006FBF7B7FA4A
S31508007A4010210920C006FBF7B2FA01211548FBF7F9
S31508007A50AEFA21E012482030807E06280ED1802119
S31508007A600920C006FBF7A3FA10210920C006FBF778
S31508007A709EFA01210B48FBF79AFA0DE080210920AE
S31508007A80C006FBF796FA01210648FBF792FA102181
S31508007A900920C006FBF78DFA00BF00BF00BF3DE70F
S31508007AA00C040020000400480C0200203075000079
S31508007AB0FCF702FAFBF748FDFBF786FEFAF77EFFAE
S31508007AC0FAF716FD0B20FAF745FC0C20FAF742FCEC
S31508007AD00920FAF73FFC0320FAF73CFC01219348FA
S31508007AE0FAF7ACFD4B200002FAF7CEFE01219048CA
S31508007AF041710021C17100208D492031C8758875F2
S31508007B0001218B488172FBF753FDFCF70BFA1A210A
S31508007B106320FCF735FAFFF759FAFCF70FFD00F07A
S31508007B20A1F9834890384089002801D1FCF74CFE1A
S31508007B307F217E20FDF7FAF800217D48C1700020DC
S31508007B407B4920318873EFE07948C0780300FDF758
S31508007B5040F90805134D8B9EB1C4D7EAFAF796FD8E
S31508007B60FFF7D4FEFDF726FFFBF722FD01F0D8FC50
S31508007B707E20FDF79DF8D6E0002301221946184617
S31508007B8000F09AFC00231A461946184600F094FCA1
S31508007B90684840686849884204D908216748FBF75D
S31508007BA006FA1DE063494868FF21F531F9F7B2FE88
S31508007BB0C007C00F00280ED180210920C006FBF798
S31508007BC0F6F910210920C006FBF7F1F901215B48F7
S31508007BD0FBF7EDF904E010210920C006FBF7E9F9E7
S31508007BE0FAF7FEFD7E20FDF763F89CE0FAF74EFDF6
S31508007BF0FBF7DEFC002301221946184600F05CFC60
S31508007C0000231A461946184600F056FC49484068AB
S31508007C104949884204D908214848FBF7C8F91DE0B4
S31508007C2044494868FF21F531F9F774FEC007C00FCB
S31508007C3000280ED180210920C006FBF7B8F91021CB
S31508007C400920C006FBF7B3F901213C48FBF7AFF959
S31508007C5004E010210920C006FBF7ABF9FEF7E2FBAA
S31508007C607E20FDF725F85EE0FDF7A0FA2021092021
S31508007C70C006FBF79EF9FAF709FDFFF747FEFDF781
S31508007C8099FEFBF795FC7E20FDF712F84BE0FDF711
S31508007C901BFC20210920C006FBF78BF9FAF7F6FC36
S31508007CA0FFF734FEFDF786FEFBF782FC7E20FCF725
S31508007CB0FFFF38E0FDF77AFA20210920C006FBF716
S31508007CC078F9FAF7E3FCFFF721FEFDF773FEFBF7F9
S31508007CD06FFC7E20FCF7ECFF25E0FDF7F5FB202185
S31508007CE00920C006FBF765F9FAF7D0FCFFF70EFE88
S31508007CF0FDF760FEFBF75CFC7E20FCF7D9FF12E07F
S31508007D00FDF76EFD20210920C006FBF752F9FAF7A8
S31508007D10BDFCFFF7FBFDFDF74DFEFBF749FC7E209A
S31508007D20FCF7C6FF00BF00BF0EE7000000240140B5
S31508007D300C0400200C020020204E0000000400481D
S31508007D40FEB546480088FAF7A4F80746444881690C
S31508007D503846FAF757F900D2FEBD414A116850680D
S31508007D60F9F777FE3E4988600A46D1689068F9F7C0
S31508007D7070FE02903A48C16801208007F9F771FE43
S31508007D800090374881680098F9F767FE0746344837
S31508007D9001693846F9F70CFE0446314948690299E3
S31508007DA0F9F75FFE01902E4A91695069F9F759FE75
S31508007DB007462B48C1693846F9F790FE0546284814
S31508007DC081682846F9F74DFE0546254A116A506925
S31508007DD0F9F747FE0746224881693846F9F77EFED5
S31508007DE0064621463046F9F73CFE064629460198DE
S31508007DF0F9F7DEFD07463146F9F7DAFD1849486214
S31508007E002A20085EFAF73AF800901548416A009861
S31508007E10F9F7CEFD0746FAF765F800B21049488526
S31508007E202A20085E898D884204DD0D48808D00B2BF
S31508007E300B4948850A482A21415E002902DA0020B2
S31508007E40074948850648C0680549086108468068A4
S31508007E50C86000200149088000BF7DE75001002066
S31508007E604804002010B540210F48F9F796FD402137
S31508007E700D48FAF787FE06210B48FDF784F90A49EB
S31508007E80898988420AD108483038008E07498842CD
S31508007E9008D0FFF7F5FCFCF72BFF03E0FFF7F0FC33
S31508007EA0FCF726FF10BD00007C030020FBAA00009B
S31508007EB0F7B5A0B00C46154680216846F9F76DFD62
S31508007EC0002700267E2168460170FE214170EF21B9
S31508007ED081700721C1702099017100214171847157
S31508007EE02112C1710121017245722912817201267E
S31508007EF005E06846805DC019C7B2701CC6B20B2E75
S31508007F00F7DBF843401CC1B26846C1727E21017393
S31508007F100D21FCF77BFB23B0F0BDFFB5A1B00646EB
S31508007F201C462A9F802101A8F9F737FD00200090FA
S31508007F3000257E21684601714671229981710721C3
S31508007F40C171239901720021417284722112C17292
S31508007F5001210173477339128173012507E001A8CE
S31508007F60415D00980818C0B20090681CC5B20B2D78
S31508007F70F5DB0098C043401CC1B26846C1737E2138
S31508007F8001740D2101A8FCF741FB25B0F0BDFFB532
S31508007F9085B005460E460E9F00200190029003907C
S31508007FA00490009000247E2168460171457186710F
S31508007FB00421C171079901720899417287723912B1
S31508007FC0C172012407E001A8015D00980818C0B233
S31508007FD00090601CC4B2082CF5DB0098C043401C16
S31508007FE0C1B2684601737E2141730A2101A8FCF7D4
S31508007FF00DFB09B0F0BD7FB5044600200090019046
S3150800800002900390002600257E2168460170FE2115
S3150800801041708F2181700321C17000210171447163
S3150800802021128171012505E06846405D8019C6B2B6
S31508008030681CC5B2072DF7DBF043401CC1B2684681
S31508008040C1717E2101720921FCF7E0FA7FBDF7B5FF
S3150800805084B005460E4600200090019002900390D9
S31508008060002700247E21684601704670857001212C
S31508008070C170694606980871012405E06846005DE6
S31508008080C019C7B2601CC4B2052CF7DBF843401C04
S31508008090C1B2684641717E2181710721FCF7B6FAA3
S315080080A007B0F0BDF0B5ABB0074680210BA8F9F7CD
S315080080B074FC0020089009900A9005900690079095
S315080080C000260490DFA00490002400253B00FCF75E
S315080080D080FE06044BC3F1EFEEEDFBF717FA0446F4
S315080080E00020089009900A90E0B22104090E2202A5
S315080080F0120E230E009201910290D4A2092108A81B
S31508008100FCF736FE7E2108A801730021417344213D
S3150800811081731321C1731522D1490CA8F9F724FCE0
S31508008120082208A90EA80330F9F71EFCC5A004907A
S3150800813005220CA803300499F9F716FC012004E07F
S315080081400BA9095C4919CDB2401C1728F8DBE8438E
S31508008150401CC1B210A8C17019267E2101711921CF
S315080081600BA8FCF753FA69E1FBF7D0F9044600209F
S31508008170089009900A90E0B22104090E2202120E14
S31508008180230E009201910290B0A2092108A8FCF7DB
S31508008190EFFDFBF7C1F9044600200590069007900D
S315080081A0E1B22004000E2202120E230E0092029162
S315080081B00190A6A2092105A8FCF7DAFD7E2108A8E8
S315080081C00173FE214173442181733321C173362221
S315080081D0A4490CA8F9F7C8FB9AA0049005220CA894
S315080081E003300499F9F7C0FB96A00490052212A85B
S315080081F00499F9F7B9FB93A00490042213A8033055
S315080082000499F9F7B1FB082208A90EA80330F9F773
S31508008210ABFB042110A8C170082205A91330F9F791
S31508008220A3FB082208A916A80330F9F79DFB01202D
S3150800823004E00BA9095C4919CDB2401C3728F8DBC4
S31508008240E843401CC1B218A8C1707E2101713921CA
S315080082500BA8FCF7DBF9F1E07E2108A80173FE21E3
S315080082604173CF2181730621C1730021017475A062
S31508008270049005220CA801300499F9F775FB012032
S3150800828004E00BA9095C4919CDB2401C0A28F8D3A9
S31508008290E843401C052149000BAA50547E210B20B7
S315080082A011540C210BA8FCF7B1F9C7E0C5E057E05B
S315080082B02BE0FFE77E2108A80173FE214173CE213A
S315080082C081730821C1730021017467A004900722F5
S315080082D00CA801300499F9F747FB012004E00BA923
S315080082E0095C4919CDB2401C0C28F8D3E843401C58
S315080082F0C1B20C200BAA11547E210D20115407205F
S3150800830041000BA8FCF782F998E07E2108A80173C2
S31508008310FE214173CD2181730821C17300210174A7
S3150800832051A0049007220CA801300499F9F71CFB08
S31508008330012004E00BA9095C4919CDB2401C0C28A0
S31508008340F8D3E843401CC1B20C200BAA11547E2175
S315080083500D201154072041000BA8FCF757F96DE0D2
S31508008360FBF7D4F804460020089009900A90E0B27A
S315080083702104090E2202120E230E00920191029088
S3150800838032A2092108A8FCF7F3FCFBF7C5F8044656
S315080083900020059006900790E1B22004000E220204
S315080083A0120E230E00920291019028A2092105A817
S315080083B0FCF7DEFC7E2108A80173FE214173CB2160
S315080083C0817300210174012141741EA004900522C5
S315080083D00CA803300499F9F7C7FA0C260BA98819D3
S315080083E0082205A9F9F7C0FA08360BA98819082240
S315080083F008A9F9F7B9FA0836701FC1B208A8C173F7
S31508008400C07B801EC1B208A88174012004E00BA9B4
S31508008410095C4919CDB2401CB042F8DBE843401C60
S315080084200BA98855701CC6B27E208855701CC6B22A
S3150800843031460BA8FCF7EAF800E000BF00BF2BB0F6
S31508008440F0BD00005350726F42000000252E3258CE
S31508008450252E3258252E3258252E32580000000077
S31508008460A6010020BB010020425F5631305F340070
S31508008470F8B506460C46F9F7DDFE051E0F4600D090
S315080084800120014349000B484908411AC90F0DD07C
S31508008490002E01D0012100E000210C4361004908AB
S315080084A0401AC00F02D10120FCF7EEFC28463946D7
S315080084B0F8BD00000000F07F0FB591B000201090C5
S315080084C00F900E900D900C90FE480078642803D00B
S315080084D0FD48407A642804D10121FB4820380172FE
S315080084E003E00021F848203801721398002802D0CA
S315080084F001287DD173E21498002803D10021F2489F
S315080085002038C172F148C1891298814203D1EF48D7
S31508008510C08A0F9001E005200F900F98052802DC0D
S3150800852005200F9004E00F98322801DB05200F90F4
S315080085300F991298411A1198814222DDE248203893
S31508008540C07A002815D1E14870384068DF4970398B
S31508008550C8611498012804D10121DB482038C1726A
S3150800856056E01498002853D10021D7482038C17204
S315080085704EE0149800284BD10021D3482038C17208
S3150800858046E00F99129841181198814240DCCE486E
S315080085902038C07A01283BD1CB48C07A012831D18E
S315080085A0CA4870384068C9497039C969401AC84903
S315080085B088420DD2C448B0380089462822DDC24810
S315080085C0B0380089801E81B2BF48B038018119E0F1
S315080085D0BE4870384068BD497039C969401A7D215E
S315080085E0890188420ED9B848B03800895F2800E06A
S315080085F0FEE307DAB448B0380089801C81B2B24875
S31508008600B03801810121B048C17200212038C172F9
S31508008610AD482038C07A01287ED1AB48807E042830
S3150800862003D0A948807E052804D1002201210846E6
S31508008630FEF712F80F991298411A119881426CDDCB
S31508008640A248703840687D21C900884207D2642054
S315080086509C49087000219C4820388173B8E19A48E3
S315080086602038807B00286DD10121974820388173F6
S315080086709648808964285CDA93486038018E408F72
S31508008680081A81B2904860388187808F0990F9F777
S3150800869000FC01460A908F480068F9F71FFA0B900C
S315080086A0F9F76CFC8C4A03C2874820380088404397
S315080086B00990F9F7F5FB0B910A9087480CC80A98B8
S315080086C0F9F7FCFA844A03C2834903C9FFF7D0FEC7
S315080086D00B910A90F9F77AFC804908607A482038A5
S315080086E000880890F9F7D5FB014609907B48006891
S315080086F0F9F7F4F97A490A90F9F7B3F90B90F9F70B
S315080087000AFC784908700846007864280DDC714828
S315080087100068F9F733FC01E057E16CE00022724B80
S315080087200B910A90F9F73EFC06D864206D4908704B
S3150800873002E064206B49087063486038018E403057
S31508008740C18245E161487038806C7D21C900884244
S315080087504CD900205D4970398864624800786428DD
S315080087603FDA59486038018E4030C08A814233DD8D
S315080087700121890757480068F9F71AF90B90F9F7A4
S31508008780CAFB81B250486038028E4030C08A101A3F
S31508008790814205DA53480078801E5249087020E065
S315080087A049486038018E4030C08A081A0A90F9F79D
S315080087B065FB0B90474801680B98F9F723FC10D224
S315080087C048480078801C474908700846007864289D
S315080087D007DD6420087004E042480078401D4149DE
S315080087E0087039486038018E4030C1823D480078AB
S315080087F034490870ECE03448C07A002876D133480A
S315080088008089642803DB64202E490870E0E02F483D
S31508008810703840687D21C900884207D264202949FA
S3150800882008700021284820388173D1E0264820386E
S31508008830807B002874D1012123482038817323487E
S315080088408089642863DA20486038018E408F081AC8
S3150800885081B21D4860388187808F0990F9F719FB26
S3150800886001460A901B480068F9F738F90B90F9F7A2
S3150800887085FB194A03C214482038008840430990EA
S31508008880F9F70EFB0B910A9013480CC80A98F9F7EA
S3150800889015FA114A03C2104903C9FFF7E9FD0B91FE
S315080088A00A90F9F793FB0D490860074820380088B5
S315080088B00890F9F7EEFA0146099008480068F9F7B2
S315080088C00DF914E0F20000202C0400207C020020A0
S315080088D070170000D4000020D8000020E000002017
S315080088E00000C842F10000200000F03F67E0FE49A2
S315080088F00A90F9F7B6F80B90F9F70DFBFB490870E3
S3150800890008460078642805DD6420087002E06420C3
S31508008910F6490870F648018E4030C18258E0FFE7F4
S31508008920F448806C7D21C900884243D90020F1496A
S315080089308864EF48018E4030C08A814231DD0121CA
S315080089408907ED480068F9F733F80B90F9F7E3FA69
S3150800895081B2E748028E4030C08A101A814205DA91
S31508008960E2480078801EE14908701FE0E048018E61
S315080089704030C08A081A0A90F9F780FA0B90DE4848
S3150800898001680B98F9F73EFB10D2D8480078801C8E
S31508008990D649087008460078642807DD6420087000
S315080089A004E0D2480078401DD0490870D048018EAE
S315080089B04030C182CD480078D049087008E0CC48DC
S315080089C05038007ACD49087002E00020CB4908707B
S315080089D0CA48027814991398FDF73EFE08E21498DF
S315080089E0002803D10021C24840300173C0486030D6
S315080089F0807E012804D002287ED003287DD199E004
S31508008A00BC48703041881298814204D1B948703008
S31508008A10408A0F9001E00A200F90B64840687D21F1
S31508008A20C900884277D3B2484030407B002872D1CB
S31508008A30AF4840300188818301214173808B0A90B9
S31508008A40F9F727FAAE490B90F9F7DCFA1AD8A848CD
S31508008A504030808B0790F9F71CFA01460890A94820
S31508008A60F9F73CF8A8490990F8F7FBFFA7490A90D7
S31508008A70F8F79EFF0B90F9F74EFAC1B29C486030A2
S31508008A8081723FE09A484030808BFF210A31884244
S31508008A901ADC97484030808B0790F9F7FAF90146B7
S31508008AA008909748F9F71AF897490990F8F7D9FFFF
S31508008AB096490A90F8F77CFF0B90F9F72CFAC1B2A1
S31508008AC08B48603081721DE089484030808B079062
S31508008AD0F9F7DFF9014608908948F8F7FFFF8C494E
S31508008AE00990F8F7BEFF89490A90F8F761FF0B90DD
S31508008AF0F9F711FAC1B202E00EE029E00BE07C4872
S31508008B00603081727A486030807A642803DB642199
S31508008B1077486030817229E076487030418812982B
S31508008B20814204D173487030408A0F9001E00A20D0
S31508008B300F901BE06F48703081881298814204D1EB
S31508008B406C487030808A0F9001E00A200F900DE083
S31508008B506848703081881298814204D1654870301F
S31508008B60808A0F9001E00A200F9000BF00BF0F987F
S31508008B70052802DC05200F9004E00F98322801DB57
S31508008B8032200F905A486030007B002802D1119895
S31508008B90FDF706FD0F991298411A119881422ADBB2
S31508008BA0544840685349086200208863C86350499E
S31508008BB01198C88708464030007B00280FD11498C2
S31508008BC0012807D11E214A48603001720121203848
S31508008BD001730BE0002146484030017306E0149803
S31508008BE0002803D100214248403001730021404843
S31508008BF04030417241E10F9912984118119881420B
S31508008C00F8DC3B484030007B012809D10021384870
S31508008C104030017337484068364908620020886347
S31508008C2033486030007B0028E4D132487030408AEF
S31508008C300A280BDB2F48406A0A90F9F72AF93549C2
S31508008C400B90F8F74BFF3449086020E0294870304C
S31508008C50408A0A2810DA27487030408A07280BDD30
S31508008C602448406A0A90F9F714F92C490B90F8F74A
S31508008C7035FF294908600AE01E48406A0A90F9F754
S31508008C8008F927490B90F8F729FF2349086018487F
S31508008C904030008B0890F9F7FCF80A9014484030E9
S31508008CA0008B0790F9F7F5F808901B4801680898B3
S31508008CB0F8F7D7FE09900A99F8F7D3FE0B90F9F75B
S31508008CC05DF9184A03C20A486030807A401D05904B
S31508008CD0F9F7E6F80991089005484030008B0190AD
S31508008CE0F9F7F2F805911FE00000C842F1000020EC
S31508008CF0CC0300200C020020D4000020F200002043
S31508008D0000007A43000082430000BE420000404053
S31508008D100000B44200803B45CC0000200000FA4425
S31508008D200080BB44E80000200490FB4903C9FFF714
S31508008D309FFB03910290059B049AF9F727F8079180
S31508008D400690099B089AF8F7B9FF0B910A90F9F76C
S31508008D50F7F881B2F1488180FF387138806A0A9045
S31508008D60F9F797F8EE490B90F8F7B8FEED49086061
S31508008D70EA489030408B0890F9F78BF80A90E74854
S31508008D809030408B0790F9F784F80890E548016819
S31508008D900898F8F766FE09900A99F8F762FE0B90AC
S31508008DA0F9F7ECF8DC4A03C2DC48B030807A401D9B
S31508008DB00590F9F775F809910890D8489030408BD6
S31508008DC00190F9F781F805910490D34903C9FFF793
S31508008DD04FFB03910290059B049AF8F7D7FF07917A
S31508008DE00690099B089AF8F769FF0B910A9000E02C
S31508008DF01BE2F9F7A5F881B2C848C180FF380138E7
S31508008E008089642827DAC84880890890F9F741F8E4
S31508008E100A90C5487038406B0590F9F73AF8C34987
S31508008E200690F8F75BFE0890BF484188FF3051303E
S31508008E30008F081A0690F9F721F807900899F8F7AD
S31508008E404DFE09900A99F8F70CFEB9490B90F8F708
S31508008E5045FEB8490860B1488088642802DB642169
S31508008E60AE488180AD48C088642802DB6421AB48DF
S31508008E70C1800121A948B0300173A8489030007B11
S31508008E8000287AD0012879D1A448B030007AAA49B6
S31508008E90097888420EDA0021A048B03001722038DD
S31508008EA001730020A0497039C86400219B48B0307E
S31508008EB0417260E10F991298411A119881420EDDAC
S31508008EC096489030407B012804D19448B030817A86
S31508008ED0417250E164219148B03041724BE18F48AC
S31508008EE0B030807E0300FBF774FF06FD04098DFC95
S31508008EF0FBFD8A48B030817A41723BE18A48703876
S31508008F00806B89497039C96B401A7D21C90088422E
S31508008F104DD985487038806B83497039C8637F4856
S31508008F205030C18F119881420CDD7C4880880A3008
S31508008F3081B27A488180C088642834DB6421774806
S31508008F40C18030E00F980B9074485030C18F11984B
S31508008F50411A0B98C20F10184010401C81420EDAB5
S31508008F606E488088801C81B26C488180C0886428DD
S31508008F7019DB64216948C18015E0FDE03AE10F98E4
S31508008F800B9066485030C18F1198411A0B98C20F42
S31508008F9010184010801C814205DD60488088801EBC
S31508008FA081B25E4881805D4950311198C8875E4814
S31508008FB0703840685C497039096A401A5F498842C6
S31508008FC011DD56488088401D81B2544881808088CA
S31508008FD0642802DB64215148818053487038406810
S31508008FE05149703908624D48B030007B002804D1D9
S31508008FF04A48B030817A417203E048480179B03076
S315080090004172B7E048487038806B47497039C96B78
S31508009010401A7D21C90088424BD943487038806B75
S3150800902041497039C8633D485030C18F1198814213
S315080090300CDD3A48C0880A3081B23848C180C088F9
S31508009040642832DB64213548C1802EE00F980B90E6
S3150800905032485030C18F1198411A0B98C20F101818
S315080090604010401C81420CDA2C48C088801C81B212
S315080090702A48C180C088642817DB64212748C18034
S3150800908013E00F980B9025485030C18F1198411A5C
S315080090900B98C20F10184010801C814205DD1F482E
S315080090A0C088801E81B21D48C1801C495031119864
S315080090B0C8871D48703840681B497039096A401AC4
S315080090C01F49884215DD1548C088401D81B21348DE
S315080090D0C180C088642802DB64211048C18002E090
S315080090E034E00BE042E01048703840680E497039A9
S315080090F008620A488179B03041723BE007489030EF
S31508009100C07A01281ED100200449B03148720021D6
S315080091100248B030017218E0E80000207C03002005
S315080091200000FA44CC0000207C02002000007A44AB
S315080091300000C842D4000020F20000208813000076
S31508009140581B00001E203B49487200BF394820388A
S31508009150C07A012806D100213648417200203549D7
S31508009160087202E01E213348417200BF322131489D
S31508009170417200BF00BF41E02E48807E012829D1F8
S315080091800F9912984118119881421FDB2948B03867
S315080091900179B03041720F9912984018801E1199C2
S315080091A088420FDD24480078002822D12148B038AB
S315080091B08088401D81B21F48B038818001201E4931
S315080091C0087016E000201C49087012E000211948B2
S315080091D041720EE01748807E042803D01548807E29
S315080091E0052803D100201349487202E00A211148D4
S315080091F0417203E000210F48417200BF00BF0D48CD
S31508009200807E012808D10B48407A02460B901499B3
S315080092101398FDF721FA07E00648007A02460B90F4
S3150800922014991398FDF718FA00BF00BF109815B0E7
S3150800923000BD00002C040020F000002010B500221C
S3150800924001210846FDF708FA4C49088CF8F721FE73
S315080092504B490860FEF774FD48482030407C0028DA
S3150800926039D14848464948604448008CB42807D054
S315080092704248008CB32803D04048008CB52804D156
S3150800928001203E492031C87403E000203B492031C3
S31508009290C8743D48406E3D49884267D93748408C76
S315080092A0801E3B49098888420DDC3448408C801C66
S315080092B037490988884206DBFDF7B6FF01202F49A2
S315080092C02031487403E02D48408C3149088000203D
S315080092D02D4948664AE029482030407C01283BD180
S315080092E02C48274948602548008CE62809D0234899
S315080092F0008CFF212C31884203D02048008CE728B7
S3150800930004D101211D482030C17403E000201B4907
S315080093102031C8741C48406E1C49884226D9174813
S31508009320408C801E1A49098888420DDC1348408CF7
S31508009330801C17490988884206DBFEF70DF80220CB
S315080093400E492031487403E00C48408C10490880C7
S3150800935000200D49486609E000200B49486608497F
S3150800936048850122FE215720FEF771FE0448408DEC
S31508009370C2B201210020FDF76FF910BD0C040020D0
S3150800938048040020000034430C0200208813000023
S31508009390000100200000664330B503465A480068BD
S315080093A0181AFF24F534A04201D957480360481E0D
S315080093B0904248DD55480078002816D1881A3C287E
S315080093C005DA881A3C24201A514C207002E0002045
S315080093D04F4C20704E4800785524201A4C4C20706B
S315080093E0204600784B4C20702AE04B48007800282D
S315080093F022D14A480088401A07280ADD454C2078B9
S31508009400C40F24186410424D2C7028460078414C2D
S31508009410207042480088401A012808DD3D48007837
S31508009420401E3C4C207020460078394C20703B4842
S3150800943002800120384C207036480078344C207061
S31508009440364802805DE0481E90424CDC481C824249
S3150800945049DC2E480078012828D12F4800780028B2
S315080094602AD12E480088801A07280BDD294C207837
S31508009470C40F24186410264D2C7028460078254CF5
S3150800948020700DE025480088801A012808DB21484D
S315080094900078401E1F4C2070204600781C4C207017
S315080094A01E48028001201C4C207005E017480078F1
S315080094B0002801D1164C2070481E904205D1154847
S315080094C00078401E124C20701BE08A4205D11148D4
S315080094D00078001F0E4C207013E00E480078801F9D
S315080094E00B4C20700DE00020094C20700A4C2070AF
S315080094F00120064C207009480088824201DB074893
S3150800950002800348007830BD04010020F8000020DE
S3150800951002010020030100200A01002008010020A2
S3150800952010B5FDF7E1FA01280AD1FE484068FF2187
S31508009530F531884203D90421FB48F9F738FD10BDF7
S31508009540FA48407900287DD10021F8482030017674
S3150800955010210920C006F9F72AFD80210920C00636
S31508009560F9F725FD0121F048F9F721FD0020EF491B
S31508009570203188760023012219461846FEF79CFFFB
S3150800958000231A4619461846FEF796FFE54840682E
S31508009590FF21F531884209D2E4482030C07D0028F1
S315080095A003D10421E048F9F704FDEDE20421DE4881
S315080095B0F9F7FDFC0020DD492031C875D948406817
S315080095C0DB498842F1D9D948807A002823D120215D
S315080095D00920C006F9F7EBFCD24840687D2149010D
S315080095E0884201D2FBF7B4F80821CF48F9F7DFFC27
S315080095F00021CE48C1710020CC492031C872002113
S31508009600CA48203001730020C649486248637D2055
S315080096104001486018E0C5488079012814D1002027
S31508009620C04948600021C148C1712030C172017328
S315080096300020BC4948624863BC492031887601212C
S31508009640BA4800E013E041714021B748F9F7A6FC93
S315080096500028AAD020210920C006F9F7AAFC002074
S31508009660B249203188760121B04841718CE2AF4871
S315080096702030807E0300FBF7ACFB07057CE7F9F892
S31508009680F7F67B000021A9480173C1720172002018
S31508009690A4490864A54920310876C87520210920FF
S315080096A0C006F9F786FC0021A0482030C172017374
S315080096B000209C494862486300219C484173002366
S315080096C0012219461846FEF7F7FE00231A461946E0
S315080096D01846FEF7F1FE95484038418E0187418EBF
S315080096E08186018EC1868F4840687D21090188429E
S315080096F02BD900208F49087040218B48F9F74EFC7A
S3150800970000281AD110210920C006F9F750FC80213B
S315080097100920C006F9F74BFC01218348F9F747FCF5
S31508009720FBF716F808218048F9F741FC7E20FBF77D
S31508009730BFFA1E20F9F700F902E0002079494860CF
S3150800974004217948F9F733FC12E008217648F9F73D
S3150800975030FC74484068FF21F531884208D97348BF
S3150800976090384089002803D104216F48F9F71FFC77
S3150800977009E26E484038018EC1866A484068FF2172
S31508009780F531884204D204216748F9F712FC03E050
S3150800979004216548F9F70BFC624948687D21C90030
S315080097A0F8F7B8F823282ED25E4948687D21C90003
S315080097B0F8F7B0F8192826D95C484038018EFF38E2
S315080097C051384088814207DA58484038418EFF3878
S315080097D05138408881420DDB54482030007B0128EF
S315080097E021D100204F494860086202214F482030A5
S315080097F0817618E000204B494860086202204B49F0
S31508009800203188760FE0474948687D21C900F8F776
S3150800981081F8232807D300204249486008620221BC
S315080098204248203081763F4A70325188FF325132A1
S31508009830508E01231A46FEF73FFE00231A461946A4
S315080098401846FEF739FE9EE138484038018EC18633
S3150800985034484068FF21F531884208D2042132484D
S31508009860F9F7A7FB07E036E1C8E07DE02BE0042125
S315080098702D48F9F79CFB2B484168703000897D22FA
S31508009880D2005043814210D2264A70325188FF32A4
S315080098905132508E01231A46FEF70EFE00231A4651
S315080098A019461846FEF708FE0CE000211F4801730A
S315080098B000201C49486001211C48417203201B49AD
S315080098C0203188765FE119484038018EC186408E7E
S315080098D0FF217D31884204DC14484038008E8842D6
S315080098E00CDD0023012219461846FEF7E5FD002384
S315080098F01A4619461846FEF7DFFD34E00949486856
S315080099007D21C900F8F706F8064970314989884269
S315080099101BD2044A70329188FF325132508E01238D
S315080099201A4609E00C020020000400480C04002036
S31508009930B80B0000C4000020FEF7BEFD00231A463F
S3150800994019461846FEF7B8FD0DE09248018E418784
S3150800995000209149486000218E4840300173042058
S315080099608C49603188760EE18A48408EFF217D3128
S31508009970884203DC8748008E88420CDD00230122DA
S3150800998019461846FEF798FD00231A461946184642
S31508009990FEF792FD31E0804948687D21C900F7F756
S315080099A0B9FF7D497031098A0F3988421ED27A4A31
S315080099B07032D189774A108E01230022FEF77CFD8A
S315080099C074484030C07A012806D10023012219467E
S315080099D01846FEF771FD10E06F4A7032D1886D4A5D
S315080099E0508E01231A46FEF767FD06E000206A49F5
S315080099F048600520674960318876C4E06648406853
S31508009A00FF21F531884204D204216448F9F7D1FAD6
S31508009A100FE061484068FF21F531884209D95E4860
S31508009A2040684B21C900884203D204215B48F9F7F4
S31508009A30BEFA594840685A4988421ED2564A703278
S31508009A40D189544A108E01230022FEF735FD51486C
S31508009A504030C07A012806D100230122194618464B
S31508009A60FEF72AFD36E04C4A7032D188494A508EB4
S31508009A7001231A46FEF720FD2CE004214748F9F792
S31508009A8098FA454840684649C831884222D300209A
S31508009A90414948603F486030807D012804D106204E
S31508009AA03C496031887605E000213A486030817685
S31508009AB0203841710023012219461846FEF7FCFC9E
S31508009AC000231A4619461846FEF7F6FC04213348C1
S31508009AD0F9F76DFA57E000212E4840300173C1723C
S31508009AE0017200202C4908640865C86400212948C9
S31508009AF06030C17520210920C006F9F75AFA0020FE
S31508009B0024496031C87208732349486248630021B2
S31508009B102048403041730023012219461846FEF7B3
S31508009B20CBFC00231A4619461846FEF7C5FC194809
S31508009B30418E0187418E8186018EC1864030C0796B
S31508009B4000281FD114484068164988421AD9FAF7DE
S31508009B50FFFD0020104948600E4850384088032809
S31508009B6008DA0C48408E5A280CDC01200949603175
S31508009B70887607E000200749603188760021054885
S31508009B804030417100BF00BF7E20FBF791F800BF4F
S31508009B90D5E40000CC0300200C0200200004004895
S31508009BA0A438000060EA0000C89B0008C80000202E
S31508009BB044010000FC220008189C00080C02002042
S31508009BC0A4080000784E0008015E2D010203040473
S31508009BD03506070809ACA24A041A5916011129259F
S31508009BE00A450181580B1058594C4C30313132789E
S31508009BF0010B11CB7E153E040132050513381206FA
S31508009C0014594132303035323848343530343241DF
S30D08009C1020041B7D5D7E0000A7
S705080018C515
